:100000000C943F080C94B64B0C94E74B0C94184C92
:100010000C94494C0C947A4C0C94AB4C0C94DC4CE6
:100020000C940D4D0C9460080C9460080C946008BE
:100030000C9460080C9460080C9460080C946008A0
:100040000C9460080C942E090C9460080C946008C1
:100050000C9460080C9460080C9433330C94E64EB6
:100060000C9460080C946F340C9460080C94600835
:100070000C9460080C9460080C9460080C94600860
:100080000C9460080C9460080C9460080C94600850
:100090000C9460080C9460080C9460080C94600840
:1000A0000C9460080C9460080C9460080C94600830
:1000B0000C9460080C9460080C9460080C94600820
:1000C0000C9460080C9460080C9460080C94600810
:1000D0000C9460080C9460080C9460080C94600800
:1000E0000C946008084AD73B3BCE016E84BCBFFD30
:1000F000C12F3D6C74319ABD56833DDA3D00C77FF8
:1001000011BED9E4BB4C3E916BAAAABE0000008090
:100110003F05A84CCDB2D44EB93836A9020C50B91F
:10012000918688083CA6AAAA2ABE000000803F65E6
:1001300063686F3A00656E6473746F7073206869EA
:10014000743A200020583A0020593A00205A3A00C8
:1001500024F404D9201BC40C5C0E9804C4095F026B
:1001600065077101F405F900FB04B300480487003A
:10017000C10369005803550003034500BE023A005D
:100180008402310053022A002902250004022000C3
:10019000E4011C00C8011900AF0117009801140008
:1001A00084011300710110006101100051010E0063
:1001B00043010D0036010B002B010B0020010B0049
:1001C000150109000C01090003010800FB000800EB
:1001D000F3000800EB000700E4000600DE00060064
:1001E000D8000600D2000600CC000500C7000500BC
:1001F000C2000500BD000400B9000400B500040001
:10020000B1000400AD000400A9000400A500030033
:10021000A20003009F0004009B000300980003005D
:100220009500020093000300900003008D0002007F
:100230008B00030088000200860002008400030097
:10024000810002007F0002007D0002007B000200AE
:1002500079000200770001007600020074000200BD
:1002600072000100710002006F0002006D000100C9
:100270006C0002006A0001006900020067000100D2
:1002800066000100650001006400020062000100D8
:1002900061000100600001005F0002005D000100DC
:1002A0005C0001005B0001005A00010059000100E0
:1002B00058000100570001005600010055000100E0
:1002C00054000100530000005300010052000100DF
:1002D00051000100500001004F0001004E000000DD
:1002E0004E0001004D0001004C0001004B000000D9
:1002F0004B0001004A0001004900010048000000D5
:1003000048000100470001004600000046000100CF
:1003100045000000450001004400010043000000CA
:1003200043000100420000004200010041000000C3
:1003300041000100400001003F0000003F000100BB
:100340003E0000003E0001003D0000003D000100B5
:100350003C0000003C0000003C0001003B000000AD
:100360003B0001003A0000003A00010039000000A3
:10037000390001003800000038000000380001009A
:100380003700000037000100360000003600000092
:100390003600010035000000350000003500010086
:1003A000340000003400000034000100330000007D
:1003B0003300000033000100320000003200000072
:1003C0003200010031000000310000003100010066
:1003D0003000000030000000300001002F0000005D
:1003E0002F0000002F0000002F0001002E00000051
:1003F0002E0000002E0001002D0000002D00000046
:100400002D0000002D0001002C0000002C00000039
:100410002C0000002C0001002B0000002B0000002D
:100420002B0000002B0001002A0000002A00000021
:100430002A0000002A000100290000002900000015
:100440002900000029000000290001002800000008
:1004500028000000280000002800000028000100FB
:1004600027000000270000002700000027000000F0
:1004700027000100260000002600000026000000E2
:1004800026000000260001002500000025000000D5
:1004900025000000250000002500000025000100C7
:1004A00024000000240000002400000024000000BC
:1004B00024000100230000002300000023000000AE
:1004C000230000002300000023000000230001009F
:1004D0002200000022000000220000002200000094
:1004E0002200000022000100210000002100000085
:1004F0002100000021000000210000002100000078
:100500002100010020000000200000002000000069
:10051000200000002000000020000000200000005B
:10052000200001001F0000001F0000001F0000004D
:100530001F0000001F0000001F0000001F0001003E
:100540001E0000001E0000001E0000001E00000033
:1005500024F4D43050C38E20C2A24017828B701175
:10056000127A910D816CD90AA861E108C758660713
:10057000615143061E4B5D05C145A7041A41110494
:10058000093D9803713931034036DB02653391022E
:10059000D4305402802E1D02632CEE01752AC50151
:1005A000B028A001102781018F2564012B244B0165
:1005B000E0223401AC211F018D200D01801FFC00C1
:1005C000841EED00971DDF00B81CD200E61BC6009C
:1005D000201BBC00641AB200B219A8000A19A000BE
:1005E0006A189900D117910040178B00B516840046
:1005F00031167E00B31579003A157300C7146F00E9
:1006000058146A00EE1366008813630025135E0019
:10061000C7125B006C12570015125400C111510033
:1006200070114F0021114B00D61049008D1047006A
:100630004610440002104200C00F4000800F3E00F0
:10064000420F3C00060F3B00CB0E3800930E3700E4
:100650005C0E3500270E3400F30D3200C10D310061
:10066000900D3000600D2E00320D2D00050D2C0078
:10067000D90C2B00AE0C2900850C29005C0C27003E
:10068000350C27000E0C2600E80B2400C40B2400B8
:10069000A00B23007D0B23005A0B2100390B2100F6
:1006A000180B2000F80A1F00D90A1E00BB0A1E0002
:1006B0009D0A1D00800A1D00630A1C00470A1B00DA
:1006C0002C0A1B00110A1A00F7091A00DD0919008B
:1006D000C4091900AB091900920917007B09180019
:1006E000630917004C091600360916002009160088
:1006F0000A091500F5081500E0081400CC081400DC
:10070000B8081400A4081400900813007D08120013
:100710006B08130058081200460812003408110034
:10072000230811001208110001081100F007100041
:10073000E0071000D0071000C0071000B0070F003E
:10074000A107100091070E0083070F0074070F0028
:1007500065070E0057070E0049070E003B070D0006
:100760002E070E0020070D0013070D0006070D00D1
:10077000F9060C00ED060D00E0060C00D4060C0096
:10078000C8060C00BC060C00B0060C00A4060B004A
:1007900099060C008D060B0082060B0077060B00F5
:1007A0006C060B0061060A0057060B004C060A0097
:1007B00042060A0038060A002E060A0024060A002D
:1007C0001A060A001006090007060A00FD050900BE
:1007D000F4050900EB050900E2050900D905090047
:1007E000D0050900C7050900BE050900B5050800C8
:1007F000AD050800A50509009C0508009405080042
:100800008C050800840508007C05080074050800B4
:100810006C050700650508005D0507005605080022
:100820004E0507004705070040050800380507008A
:10083000310507002A050700230507001C050600EF
:10084000160507000F05070008050600020507004A
:10085000FB040600F5040700EE040600E8040600A9
:10086000E2040700DB040600D5040600CF040600FE
:10087000C9040600C3040600BD040600B704060050
:10088000B1040500AC040600A6040600A00405009F
:100890009B04060095040500900406008A040500E8
:1008A00085040500800406007A040500750405002F
:1008B000700405006B040500660405006104050072
:1008C0005C04050057040500520405004D040500B2
:1008D00048040500430405003E0404003A040500F2
:1008E00035040500300404002C040500270404002E
:1008F000230405001E0404001A0404001604050065
:10090000110404000D04040009040500040404009B
:1009100000040400FC030400F8030400F4030400D2
:10092000F0030400EC030400E8030400E403040003
:10093000E0030400DC030400D8030400D403040033
:10094000D0030400CC030400C8030300C503030064
:100950006563686F3A00656E717565696E67202220
:10096000002200737461727400506F776572557065
:10097000002045787465726E616C205265736574F1
:10098000002042726F776E206F7574205265736518
:100990007400205761746368646F672052657365E3
:1009A000740020536F6674776172652052657365B9
:1009B00074004D61726C696E3A2000312E302E3019
:1009C0002052433200204C6173742055706461746E
:1009D00065643A20004D61726C696E2D4D6F6E2C0E
:1009E0002035204D617220323031322030393A3595
:1009F000363A3530202D30383030202D20663330D7
:100A000039353439336230366435326133336165B8
:100A100037376130623863316639326132323633AA
:100A2000333236316100207C20417574686F723A30
:100A300020004275696C642D4D652D4D61726C69A5
:100A40006E002046726565204D656D6F72793A20A3
:100A5000002020506C616E6E65724275666665722C
:100A600042797465733A200053746F726564207321
:100A7000657474696E6773207265747265697665F2
:100A8000643A0053746570732070657220756E69E6
:100A9000743A0020204D3932205800205900205A45
:100AA000002045004D6178696D756D20666565644F
:100AB000726174657320286D6D2F73293A002020B0
:100AC0004D323033205800205900205A0020450074
:100AD0004D6178696D756D20416363656C65726108
:100AE00074696F6E20286D6D2F7332293A002020B3
:100AF0004D323031205800205900205A0020450046
:100B0000416363656C65726174696F6E3A20533D31
:100B1000616363656C65726174696F6E2C20543D0E
:100B20007265747261637420616363656C65726180
:100B300074696F6E0020204D3230342053002054F1
:100B400000416476616E63656420766172696162FA
:100B50006C65733A20533D4D696E2066656564721D
:100B600061746520286D6D2F73292C20543D4D69CB
:100B70006E2074726176656C20666565647261745E
:100B80006520286D6D2F73292C20423D6D696E699B
:100B90006D756D207365676D656E742074696D6524
:100BA00020286D73292C20583D6D6178696D756D15
:100BB000207859206A65726B20286D6D2F73292C5F
:100BC00020205A3D6D6178696D756D205A206A65E7
:100BD000726B20286D6D2F73290020204D32303527
:100BE000205300205400204200205800205A0020AA
:100BF00045005049442073657474696E67733A0008
:100C00002020204D33303120500020490020440066
:100C10004572726F723A004C696E65204E756D6256
:100C20006572206973206E6F74204C617374204C60
:100C3000696E65204E756D6265722B312C204C619A
:100C40007374204C696E653A00636865636B7375F5
:100C50006D206D69736D617463682C204C617374D1
:100C6000204C696E653A004E6F20436865636B7374
:100C7000756D2077697468206C696E65206E756D7E
:100C80006265722C204C617374204C696E653A0069
:100C90004E6F204C696E65204E756D6265722077CF
:100CA00069746820636865636B73756D2C204C6193
:100CB0007374204C696E653A006F6B006F6B205443
:100CC0003A0020423A0020403A00543A0020453A87
:100CD0000020573A00543A0020453A0020423A009A
:100CE0004649524D574152455F4E414D453A4D613F
:100CF000726C696E2056313B20537072696E746558
:100D0000722F6772626C206D617368757020666FF8
:100D1000722067656E36204649524D574152455FF5
:100D200055524C3A687474703A2F2F7777772E6D3E
:100D3000656E64656C2D70617274732E636F6D20C7
:100D400050524F544F434F4C5F56455253494F4EAC
:100D50003A312E30204D414348494E455F54595059
:100D6000453A4D656E64656C20455854525544456E
:100D7000525F434F554E543A310A00583A00593A9F
:100D8000005A3A00453A0020436F756E7420583A75
:100D900000593A005A3A00785F6D696E3A00785F00
:100DA0006D61783A00795F6D696E3A00795F6D61C7
:100DB000783A007A5F6D696E3A007A5F6D61783AD1
:100DC00000556E6B6E6F776E20636F6D6D616E6434
:100DD0003A2200220053657474696E67732053745D
:100DE0006F72656400526573656E643A006F6B00E4
:100DF0005072696E7465722068616C7465642E202F
:100E00006B696C6C28292063616C6C6564202121FE
:100E1000004572726F723A00202D20496E76616C27
:100E20006964206578747275646572206E756D6290
:100E300065722100202D20496E76616C6964206501
:100E400078747275646572206E756D6265722021AA
:100E5000003A2045787472756465722073776974FE
:100E600063686564206F66662E204D415854454D79
:100E700050207472696767657265642021003A20AA
:100E800045787472756465722073776974636865F8
:100E900064206F66662E204D494E54454D50207497
:100EA000726967676572656420210054656D7065BD
:100EB000726174757265206865617465642062652D
:100EC00064207377697463686564206F66662E209A
:100ED0004D415854454D502074726967676572657D
:100EE00064202121006563686F3A0020636F6C64A1
:100EF00020657874727573696F6E2070726576659F
:100F00006E7465640020746F6F206C6F6E6720656F
:100F10007874727573696F6E2070726576656E7421
:100F20006564000000090A02080B0C0D07060304A3
:100F300001000000000000000000000000000000B0
:100F40000000000000000000000000000000001190
:100F5000100F000000000000000000000000000072
:100F6000000000000000000000010210202008081E
:100F700010204010204080020102010804020101FB
:100F800002040810204080804020100804020180E4
:100F9000040201804020100804020108040201013B
:100FA000020408102040800102040810204080053F
:100FB000050505070508080808020202020A0A08D2
:100FC00008040404040101010101010101030303F8
:100FD0000303030303040707070C0C0C0C0C0C0C95
:100FE0000C0202020206060606060606060B0B0B9C
:100FF0000B0B0B0B0B000020002300260029002CFC
:10100000002F003200000100000301060109010069
:10101000002200250028002B002E003100340002A1
:10102000010000050108010B010000210024002738
:10103000002A002D003000330001010000040107E8
:10104000010A01494E46494E4954594E414E00004D
:1010500020410000C84200401C4620BCBE4CCA1BB8
:101060000E5AAEC59D74CDCCCC3D0AD7233C17B7E4
:10107000D13877CC2B329595E6241FB14F0A112435
:101080001FBECFEFD1E2DEBFCDBF00E00CBF13E04B
:10109000A0E0B2E0EEEFF5EB00E00BBF02C007907E
:1010A0000D92AA36B107D9F71BE0AAE6B3E001C05A
:1010B0001D92A93EB107E1F70E94F74F0C94FD5A2B
:1010C0000C94000080917C03882349F480917B0379
:1010D000882329F480917A03882309F4AEC0EFE2D3
:1010E000F1E007C09091C00095FFFCCF8093C6004F
:1010F000319684918823B1F7E5E3F1E007C0909140
:10110000C00095FFFCCF8093C60031968491882360
:10111000B1F780917C03882349F1E4E4F1E007C052
:101120009091C00095FFFCCF8093C60031968491CA
:101130008823B1F760917D0370917E0380917F03D6
:10114000909180030E9480512091920B3091930BDB
:101150004091940B5091950B0E94E550AB01BC015E
:101160008EEE95E022E030E00E94CF3680917B0346
:10117000882349F1E8E4F1E007C09091C00095FFB1
:10118000FCCF8093C600319684918823B1F760919B
:1011900081037091820380918303909184030E9464
:1011A00080512091960B3091970B4091980B509164
:1011B000990B0E94E550AB01BC018EEE95E022E058
:1011C00030E00E94CF3680917A03882349F1ECE425
:1011D000F1E007C09091C00095FFFCCF8093C6005E
:1011E000319684918823B1F76091850370918603CD
:1011F00080918703909188030E94805120919A0BDF
:1012000030919B0B40919C0B50919D0B0E94E5509F
:10121000AB01BC018EEE95E022E030E00E94CF36BB
:101220008091C00085FFFCCF8AE08093C6001092B9
:101230007C0310927B0310927A03089510927C0332
:1012400010927B0310927A0308958093FB02089515
:10125000EFE6F0E080818260808308951F920F9214
:101260000FB60F920BB60F9211240F931F932F936B
:101270003F934F935F936F937F938F939F93AF931E
:10128000BF93CF93DF93EF93FF9380918D03909162
:101290008E03009709F082C19091750680917406C3
:1012A0009817A1F02091740630E08DE490E0289F1B
:1012B000F001299FF00D389FF00D1124EA58F94FE5
:1012C000DF01A45BBF4F81E08C9302C0E0E0F0E05F
:1012D000F0938E03E0938D03309709F459C1109277
:1012E0008F0310929003109291031092920364ADB9
:1012F00075AD70939403609393032CE96134720786
:1013000028F48EE46132780748F002C060E47CE99A
:10131000769567957695679584E007C0E7E2613139
:101320007E0730F07695679582E08093950308C03C
:1013300081E0809395036032710510F460E270E003
:1013400060527040F8E060307F07E0F0272F30E017
:10135000220F331F220F331F205B3E4FF9013296BD
:1013600085919491AA27699FE001689FC10DDA1FBA
:101370000694CA1FDA1F1124F901459154914C1BA0
:101380005D0B1FC0CB01969587958C7F805B9A4F34
:10139000FC01459154910296FC01A591B491862FD0
:1013A00090E087709070A89F9001A99F300DB89F22
:1013B000300D1124D3E036952795DA95E1F7421BDD
:1013C000530B44365105A0F4E0E0F2E006C09091E2
:1013D000C00095FFFCCF8093C60081918823B9F7A8
:1013E0008EEE95E04AE050E00E94F43544E650E08D
:1013F000CA01A0E0B0E08093960390939703A09376
:101400009803B09399035093890040938800E0912A
:101410008D03F0918E0360AD71AD2CE961347207DC
:1014200028F48EE46132780748F002C060E47CE979
:10143000769567957695679584E007C0E7E2613118
:101440007E0730F07695679582E08093950308C01B
:1014500081E0809395036032710510F460E270E0E2
:1014600060527040F8E060307F07E0F0272F30E0F6
:10147000220F331F220F331F205B3E4FF90132969C
:1014800085919491AA27699FE001689FC10DDA1F99
:101490000694CA1FDA1F1124F901459154914C1B7F
:1014A0005D0B1FC0CB01969587958C7F805B9A4F13
:1014B000FC01459154910296FC01A591B491862FAF
:1014C00090E087709070A89F9001A99F300DB89F01
:1014D000300D1124E3E036952795EA95E1F7421B9C
:1014E000530B44365105A0F4E0E0F2E006C09091C1
:1014F000C00095FFFCCF8093C60081918823B9F787
:101500008EEE95E04AE050E00E94F43544E650E06B
:1015100050939B0340939A03E0918D03F0918E03C7
:1015200080899189A289B389B695A7959795879562
:10153000B095A095909581959F4FAF4FBF4F8093E9
:101540009C0390939D03A0939E03B0939F0380936D
:10155000A0039093A103A093A203B093A30380934D
:10156000A4039093A503A093A603B093A70380932D
:10157000A8039093A903A093AA03B093AB0310927E
:10158000890310928A0310928B0310928C0306C079
:1015900080ED97E09093890080938800E0918D031F
:1015A000F0918E03309709F41AC580A18093AC03A3
:1015B00080FF37C0119A8FEF8093F70220B121701E
:1015C00031E0232759F18091AD03882339F18081DF
:1015D0009181A281B381181619061A061B06F4F42C
:1015E00080916A0390916B03A0916C03B0916D039D
:1015F00080937D0390937E03A0937F03B093800339
:1016000030937C0380899189A289B389809389036F
:1016100090938A03A0938B03B0938C032093AD0324
:1016200036C0119881E08093F70221E0029B02C04E
:1016300020E02BC08091AE03882339F18081918115
:10164000A281B381181619061A061B06F4F48091BC
:101650006A0390916B03A0916C03B0916D0380932A
:101660007D0390937E03A0937F03B0938003209328
:101670007C0380899189A289B3898093890390939F
:101680008A03A0938B03B0938C032093AE038091C5
:10169000AC0381FF3BC044988FEF8093F80221E0B8
:1016A000049B02C020E02FC08091AF03882359F132
:1016B000E0918D03F0918E0384819581A681B7819D
:1016C000181619061A061B06F4F480916E03909101
:1016D0006F03A0917003B091710380938103909385
:1016E0008203A0938303B093840320937B038089B8
:1016F0009189A289B3898093890390938A03A093E7
:101700008B03B0938C032093AF033AC0449A81E0DB
:101710008093F80221E0069B02C020E02FC0809158
:10172000B003882359F1E0918D03F0918E038481F9
:101730009581A681B781181619061A061B06F4F4BE
:1017400080916E0390916F03A0917003B09171032B
:101750008093810390938203A0938303B0938403C7
:1017600020937B0380899189A289B389809389031F
:1017700090938A03A0938B03B0938C032093B003C0
:101780008091AC0382FF3DC0A29A8FEF8093F90253
:1017900026B12095221F2227221F81F18091B103BB
:1017A000882361F1E0918D03F0918E03808591850E
:1017B000A285B385181619061A061B06FCF480913B
:1017C000720390917303A0917403B0917503809399
:1017D000850390938603A0938703B093880381E0E9
:1017E00080937A0380899189A289B3898093890340
:1017F00090938A03A0938B03B0938C032093B1033F
:101800003AC0A29881E08093F90221E0359B02C0A2
:1018100020E02FC08091B203882359F1E0918D031D
:10182000F0918E0380859185A285B38518161906DF
:101830001A061B06F4F48091720390917303A09131
:101840007403B09175038093850390938603A093EE
:101850008703B093880320937A0380899189A289B2
:10186000B3898093890390938A03A0938B03B093E9
:101870008C032093B2038091AC039FB7F89483FF4D
:1018800008C080910B018F7E80930B019FBF8FEF6B
:1018900007C080910B01806180930B019FBF81E0A5
:1018A0008093FA02C0E0D0E086C18091C00087FF3B
:1018B0001AC06091C60080916F0690917006AC01CD
:1018C0004F5F5F4F4F7750702091710630917206D5
:1018D0004217530741F081519A4FFC0160835093A6
:1018E000700640936F06E0918D03F0918E03409156
:1018F0009C0350919D0360919E0370919F03808192
:101900009181A281B381480F591F6A1F7B1F4093A9
:101910009C0350939D0360939E0370939F03141642
:1019200015061606170644F5139A80899189A2892F
:10193000B389481B590B6A0B7B0B40939C03509354
:101940009D0360939E0370939F03139880916A0395
:1019500090916B03A0916C03B0916D032091F702FD
:10196000820F911DA11DB11D80936A0390936B039B
:10197000A0936C03B0936D03E0918D03F0918E03FF
:101980004091A0035091A1036091A2037091A30321
:1019900084819581A681B781480F591F6A1F7B1FDB
:1019A0004093A0035093A1036093A2037093A303F9
:1019B000141615061606170644F5469A808991896D
:1019C000A289B389481B590B6A0B7B0B4093A00378
:1019D0005093A1036093A2037093A3034698809150
:1019E0006E0390916F03A0917003B09171032091E9
:1019F000F802820F911DA11DB11D80936E0390937B
:101A00006F03A0937003B0937103E0918D03F09185
:101A10008E034091A4035091A5036091A603709199
:101A2000A70380859185A285B385480F591F6A1F3A
:101A30007B1F4093A4035093A5036093A603709368
:101A4000A703141615061606170644F5409A808952
:101A50009189A289B389481B590B6A0B7B0B409370
:101A6000A4035093A5036093A6037093A703409823
:101A70008091720390917303A0917403B0917503E8
:101A80002091F902820F911DA11DB11D8093720357
:101A900090937303A0937403B0937503E0918D0347
:101AA000F0918E038091A8039091A903A091AA03BD
:101AB000B091AB034485558566857785840F951F66
:101AC000A61FB71F8093A8039093A903A093AA030E
:101AD000B093AB03181619061A061B060CF042C089
:101AE0009FB7F89480910B01806480930B019FBF96
:101AF000E0918D03F0918E038091A8039091A9034A
:101B0000A091AA03B091AB0340895189628973897E
:101B1000841B950BA60BB70B8093A8039093A90386
:101B2000A093AA03B093AB039FB7F89480910B01E5
:101B30008F7B80930B019FBF8091760390917703F9
:101B4000A0917803B09179032091FA02820F911D40
:101B5000A11DB11D8093760390937703A093780322
:101B6000B09379038091890390918A03A0918B03AC
:101B7000B0918C030196A11DB11D809389039093B0
:101B80008A03A0938B03B0938C0380918903909177
:101B90008A03A0918B03B0918C032196E0918D0371
:101BA000F0918E0340895189628973898417950762
:101BB000A607B70738F48091950390E0C817D907B6
:101BC0000CF473CE4091890350918A0360918B038A
:101BD00070918C03E0918D03F0918E038489958937
:101BE000A689B78984179507A607B70708F4DCC04C
:101BF00000919603109197032091980330919903D7
:101C0000448D558D668D778DAA27059FB12D169F22
:101C1000C001269F900D259F800D911D069FB00D40
:101C2000811D9A1F159FB00D811D9A1F249FB00D15
:101C3000811D9A1F149FB10D8A1F9A1FB6958A1F86
:101C40009A1F112424AD35AD280F391F309394030A
:101C50002093930380AD91ADA2ADB3ADA90160E037
:101C600070E084179507A607B70720F490939403B4
:101C7000809393036091930370919403FCE9613422
:101C80007F0728F42EE46132720748F002C060E456
:101C90007CE9769567957695679584E007C087E23D
:101CA0006131780730F07695679582E080939503EF
:101CB00008C081E0809395036032710510F460E202
:101CC00070E060527040E8E060307E07E0F0272F5F
:101CD00030E0220F331F220F331F205B3E4FF901EC
:101CE000329685919491AA27699FE001689FC10D62
:101CF000DA1F0694CA1FDA1F1124F9014591549185
:101D00004C1B5D0B1FC0CB01969587958C7F805B2C
:101D10009A4FFC01459154910296FC01A591B49112
:101D2000862F90E087709070A89F9001A99F300D3A
:101D3000B89F300D1124D3E036952795DA95E1F759
:101D4000421B530B44365105A0F4E0E0F2E006C01C
:101D50009091C00095FFFCCF8093C60081918823AD
:101D6000B9F78EEE95E04AE050E00E94F43544E683
:101D700050E0509389004093880060E070E08091CB
:101D8000960390919703A0919803B0919903840FC3
:101D9000951FA61FB71F8093960390939703A09358
:101DA0009803B0939903F6C04091890350918A0338
:101DB00060918B0370918C03808D918DA28DB38D7A
:101DC00084179507A607B70708F0DCC000918F03BA
:101DD000109190032091910330919203448D558D81
:101DE000668D778DAA27059FB12D169FE001269F4E
:101DF000D00D259FC00DD11D069FB00DC11DDA1F4E
:101E0000159FB00DC11DDA1F249FB00DC11DDA1F33
:101E1000149FB10DCA1FDA1FB695CA1FDA1F11240D
:101E20008091930390919403E05CFF4F8C179D0782
:101E300018F48081918102C08C1B9D0B40815181DF
:101E4000628173818C0120E030E0041715072607BA
:101E5000370708F4CA01FCE981349F0728F42EE40F
:101E60008132920748F002C080E49CE996958795FC
:101E70009695879524E007C0E7E281319E0730F010
:101E80009695879522E02093950308C021E0209342
:101E900095038032910510F480E290E0BC0160521D
:101EA0007040F8E060307F07E0F0272F30E0220F2D
:101EB000331F220F331F205B3E4FF901329685916D
:101EC0009491AA27699FE001689FC10DDA1F0694CB
:101ED000CA1FDA1F1124F901459154914C1B5D0B67
:101EE0001FC0CB01969587958C7F805B9A4FFC0134
:101EF000459154910296FC01A591B491862F90E0F2
:101F000087709070A89F9001A99F300DB89F300DE9
:101F10001124E3E036952795EA95E1F7421B530B30
:101F200044365105A0F4E0E0F2E006C09091C00014
:101F300095FFFCCF8093C60081918823B9F78EEE80
:101F400095E04AE050E00E94F43544E650E05093BA
:101F500089004093880060E070E080918F03909149
:101F60009003A0919103B0919203840F951FA61F37
:101F7000B71F80938F0390939003A0939103B09326
:101F8000920308C080919A0390919B0390938900DB
:101F9000809388004091890350918A0360918B035C
:101FA00070918C03E0918D03F0918E03808991896B
:101FB000A289B389481759076A077B0780F01092F6
:101FC0008E0310928D039091750680917406981778
:101FD00031F0809174068F5F8F7080937406FF914B
:101FE000EF91DF91CF91BF91AF919F918F917F91B1
:101FF0006F915F914F913F912F911F910F910F9092
:102000000BBE0F900FBE0F901F901895099A3C9A27
:102010009A9AEAE0F1E08081806180838081846027
:1020200080830D9A159A0F9A179A3A9A429A989A1B
:10203000A09A229A2A9A0898109A0A98129A0C98AA
:10204000149A0E98169A3F98479A3D98459A0B9A7B
:102050003E9A389A80818064808380818160808309
:10206000A1E8B0E08C918F7E8C938C9188608C93EA
:10207000E0E8F0E080818D7F808380818E7F8083A7
:1020800080818F73808380818F7C80838C91887F17
:1020900082608C9380E090E4909389008093880024
:1020A0001092850010928400EFE6F0E0808182605B
:1020B000808381E08093FB02789408959091750667
:1020C00080917406981731F00E94113081E00E94CF
:1020D000E019F4CF0895CF93DF93EFB7F894EC01B4
:1020E00088819981AA81BB8180936A0390936B0355
:1020F000A0936C03B0936D03EB0188819981AA8151
:10210000BB8180936E0390936F03A0937003B09391
:102110007103EA0188819981AA81BB81809372034E
:1021200090937303A0937403B0937503E9018881BE
:102130009981AA81BB818093760390937703A093C2
:102140007803B0937903EFBFDF91CF9108952FB754
:10215000F894FC0180819181A281B3818093760300
:1021600090937703A0937803B09379032FBF0895DA
:102170000F931F939FB7F894E82FF0E0EE0FFF1F27
:10218000EE0FFF1FE659FC4F008111812281338140
:102190009FBFB801C9011F910F9108950E945E1061
:1021A000159A179A429AA09A0895CF93DF93C0E5A3
:1021B000D9E0FE0107C09091C00095FFFCCF80934D
:1021C000C600319684918823B1F7E3E8FAE007C0AE
:1021D0009091C00095FFFCCF8093C600319684910A
:1021E0008823B1F78091C00085FFFCCF8AE08093FF
:1021F000C600FE018491E0E5F9E008C09091C000BE
:1022000095FFFCCF8093C600319684918823B1F767
:10221000E3E9FAE007C09091C00095FFFCCF8093FE
:10222000C600319684918823B1F74091920B50916A
:10223000930B6091940B7091950B8EEE95E022E0DC
:1022400030E00E94CF36EBE9FAE007C09091C00081
:1022500095FFFCCF8093C600319684918823B1F717
:102260004091960B5091970B6091980B7091990B40
:102270008EEE95E022E030E00E94CF36EEE9FAE003
:1022800007C09091C00095FFFCCF8093C6003196A7
:1022900084918823B1F740919A0B50919B0B6091E8
:1022A0009C0B70919D0B8EEE95E022E030E00E9439
:1022B000CF36E1EAFAE007C09091C00095FFFCCF6D
:1022C0008093C600319684918823B1F740919E0B8C
:1022D00050919F0B6091A00B7091A10B8EEE95E039
:1022E00022E030E00E94CF368091C00085FFFCCF15
:1022F0008AE08093C600FE018491E0E5F9E008C021
:102300009091C00095FFFCCF8093C60031968491D8
:102310008823B1F7E4EAFAE007C09091C00095FF86
:10232000FCCF8093C600319684918823B1F78091C9
:10233000C00085FFFCCF8AE08093C600FE01849137
:10234000E0E5F9E008C09091C00095FFFCCF8093D4
:10235000C600319684918823B1F7EEEBFAE007C00E
:102360009091C00095FFFCCF8093C6003196849178
:102370008823B1F74091A20B5091A30B6091A40B5D
:102380007091A50B8EEE95E022E030E00E94CF36F2
:10239000E7ECFAE007C09091C00095FFFCCF809376
:1023A000C600319684918823B1F74091A60B5091D5
:1023B000A70B6091A80B7091A90B8EEE95E022E01F
:1023C00030E00E94CF36EAECFAE007C09091C000FE
:1023D00095FFFCCF8093C600319684918823B1F796
:1023E0004091AA0B5091AB0B6091AC0B7091AD0B6F
:1023F0008EEE95E022E030E00E94CF36EDECFAE080
:1024000007C09091C00095FFFCCF8093C600319625
:1024100084918823B1F74091AE0B5091AF0B60913E
:10242000B00B7091B10B8EEE95E022E030E00E948F
:10243000CF368091C00085FFFCCF8AE08093C60034
:10244000FE018491E0E5F9E008C09091C00095FF9D
:10245000FCCF8093C600319684918823B1F7E0EDDC
:10246000FAE007C09091C00095FFFCCF8093C600B2
:10247000319684918823B1F78091C00085FFFCCF0D
:102480008AE08093C600FE018491E0E5F9E008C08F
:102490009091C00095FFFCCF8093C6003196849147
:1024A0008823B1F7EEEEFAE007C09091C00095FFE7
:1024B000FCCF8093C600319684918823B1F7409178
:1024C000820B5091830B6091840B7091850B8EEE83
:1024D00095E02AE030E00E948935E7EFFAE007C096
:1024E0009091C00095FFFCCF8093C60031968491F7
:1024F0008823B1F74091860B5091870B6091880B30
:102500007091890B8EEE95E02AE030E00E948935CB
:10251000EAEFFAE007C09091C00095FFFCCF8093EE
:10252000C600319684918823B1F740918A0B50916F
:102530008B0B60918C0B70918D0B8EEE95E02AE0E9
:1025400030E00E948935EDEFFAE007C09091C000BD
:1025500095FFFCCF8093C600319684918823B1F714
:1025600040918E0B50918F0B6091900B7091910B5D
:102570008EEE95E02AE030E00E9489358091C0001F
:1025800085FFFCCF8AE08093C600FE018491E0E5E0
:10259000F9E008C09091C00095FFFCCF8093C60081
:1025A000319684918823B1F7E0E0FBE007C0909179
:1025B000C00095FFFCCF8093C6003196849188239C
:1025C000B1F78091C00085FFFCCF8AE08093C60000
:1025D000FE018491E0E5F9E008C09091C00095FF0C
:1025E000FCCF8093C600319684918823B1F7E5E350
:1025F000FBE007C09091C00095FFFCCF8093C60020
:10260000319684918823B1F740917A0B50917B0BDE
:1026100060917C0B70917D0B8EEE95E022E030E0B6
:102620000E94CF36EEE3FBE007C09091C00095FF1B
:10263000FCCF8093C600319684918823B1F74091F6
:10264000760B5091770B6091780B7091790B8EEE31
:1026500095E022E030E00E94CF368091C00085FFF7
:10266000FCCF8AE08093C600FE018491E0E5F9E0AA
:1026700008C09091C00095FFFCCF8093C6003196B2
:1026800084918823B1F7E1E4FBE007C09091C0009A
:1026900095FFFCCF8093C600319684918823B1F7D3
:1026A0008091C00085FFFCCF8AE08093C600FE01C8
:1026B0008491E0E5F9E008C09091C00095FFFCCF5F
:1026C0008093C600319684918823B1F7EAEDFBE050
:1026D00007C09091C00095FFFCCF8093C600319653
:1026E00084918823B1F740917E0B50917F0B6091CC
:1026F000800B7091810B8EEE95E022E030E00E941D
:10270000CF36E3EEFBE007C09091C00095FFFCCF11
:102710008093C600319684918823B1F74091660B6F
:102720005091670B6091680B7091690B8EEE95E08C
:1027300022E030E00E94CF36E6EEFBE007C0909149
:10274000C00095FFFCCF8093C6003196849188230A
:10275000B1F74091B20B5091B30B6091B40B7091F3
:10276000B50B8EEE95E02AE030E00E948935E9EE67
:10277000FBE007C09091C00095FFFCCF8093C6009E
:10278000319684918823B1F74091720B5091730B6D
:102790006091740B7091750B8EEE95E022E030E045
:1027A0000E94CF36ECEEFBE007C09091C00095FF91
:1027B000FCCF8093C600319684918823B1F7409175
:1027C0006E0B50916F0B6091700B7091710B8EEED0
:1027D00095E022E030E00E94CF36EFEEFBE007C04C
:1027E0009091C00095FFFCCF8093C60031968491F4
:1027F0008823B1F740916A0B50916B0B60916C0B81
:1028000070916D0B8EEE95E022E030E00E94CF36A5
:102810008091C00085FFFCCF8AE08093C600FE0156
:102820008491E0E5F9E008C09091C00095FFFCCFED
:102830008093C600319684918823B1F7E2EFFBE0E4
:1028400007C09091C00095FFFCCF8093C6003196E1
:1028500084918823B1F78091C00085FFFCCF8AE086
:102860008093C600FE01C491E0E5F9E008C08091C4
:10287000C00085FFFCCFC093C6003196C491CC2325
:10288000B1F7E0E0FCE007C09091C00095FFFCCFFD
:102890008093C600319684918823B1F74091250337
:1028A0005091260360912703709128038EEE95E0E6
:1028B00022E030E00E94CF36EAE0FCE007C09091D1
:1028C000C00095FFFCCF8093C60031968491882389
:1028D000B1F76091210370912203809123039091BD
:1028E00024032FE632E143E05EE30E94E550AB01B2
:1028F000BC018EEE95E022E030E00E94CF36EDE0A4
:10290000FCE007C09091C00095FFFCCF8093C6000B
:10291000319684918823B1F760911D0370911E0355
:1029200080911F03909120032FE632E143E05EE3A4
:102930000E94B353AB01BC018EEE95E022E030E083
:102940000E94CF368091C00085FFFCCF8AE0809343
:10295000C600DF91CF910895CF93DF930F920F922E
:10296000CDB7DEB78091E30B9091E40B9E012F5F12
:102970003F4F009719F4295E3B4002C0281B390BDA
:102980003A83298389819A810F900F90DF91CF91AB
:102990000895809A889A0895809A889808958091D9
:1029A000660590916705019660E070E00E94FC5416
:1029B000462F572F682F792FCB01BA0108958091A8
:1029C000660590916705019660E070E04AE050E08E
:1029D0000E947B560895682FE0916005F091610593
:1029E00040E650E0E49F9001E59F300DF49F300DEC
:1029F0001124C90184529C4F70E00E94DA579C0157
:102A0000909367058093660581E02115310509F4EF
:102A100080E008950E94304FDC01CB018093700567
:102A200090937105A0937205B0937305EDEEFDE0F0
:102A300007C09091C00095FFFCCF8093C6003196EF
:102A400084918823B1F78091C00085FFFCCF8AE094
:102A50008093C60008958EEE95E00E940235E5EE63
:102A6000FDE007C09091C00095FFFCCF8093C600A9
:102A7000319684918823B1F740916C0550916D0592
:102A800060916E0570916F054F5F5F4F6F4F7F4F85
:102A90008EEE95E02AE030E00E949E358091C000E5
:102AA00085FFFCCF8AE08093C6000E940A15089536
:102AB0002F923F925F926F927F928F929F92AF92EE
:102AC000BF92CF92DF92EF92FF920F931F93CF931B
:102AD000DF9330E6832E912C44E0242E312CE9EB59
:102AE000FCE074905AE0652E55245394F6C18D3065
:102AF00031F08A3321F04F3551050CF4D0C1411526
:102B0000510519F4109265050BC28091DA0390917A
:102B1000DB03889D8001899D100D989D100D112467
:102B2000400F511F44525C4FFA01108220916505FD
:102B3000222309F0AFC110926505845A9A4FFC0117
:102B40001082E801C452DC4FCE016EE470E00E94B6
:102B5000DA57009709F410C19093670580936605D2
:102B60008C1B9D0B800F911F83529C4F60E070E087
:102B70004AE050E00E947B56DC01CB01809368055F
:102B800090936905A0936A05B0936B05C0906C059E
:102B9000D0906D05E0906E05F0906F05B701A6012D
:102BA0004F5F5F4F6F4F7F4F84179507A607B7079B
:102BB00009F43AC02091DA033091DB03289DC0016B
:102BC000299D900D389D900D112484529C4F64E1F5
:102BD00072E00E94F357009739F5E0E1FCE007C08E
:102BE0009091C00095FFFCCF8093C60031968491F0
:102BF0008823B1F7E7E1FCE007C09091C00095FFA2
:102C0000FCCF8093C600319684918823B1F78EEE75
:102C100095E0B701A6012AE030E00E949E35809140
:102C2000C00085FFFCCF91C08091DA039091DB0357
:102C3000889D8001899D100D989D100D11242CED0B
:102C4000A22E23E0B22EA00EB11EC5016AE270E0F2
:102C50000E94DA57009721F452C0C3272F5F02C0A9
:102C600020E0C0E0F801E20FF11DE452FC4F30819A
:102C70003A3299F790936705809366058A199B0904
:102C8000800F911F83529C4F60E070E00E94FC54C3
:102C90000E944D51AB01BC018C2F90E08417950729
:102CA00009F459C0E0E1FCE007C09091C00095FF35
:102CB000FCCF8093C600319684918823B1F7E9E474
:102CC000FCE007C09091C00095FFFCCF8093C60048
:102CD000319684918823B1F740916C0550916D0530
:102CE00060916E0570916F058EEE95E02AE030E000
:102CF0000E949E358091C00085FFFCCF26C0E0E198
:102D0000FCE007C09091C00095FFFCCF8093C60007
:102D1000319684918823B1F7E7E6FCE007C09091F3
:102D2000C00095FFFCCF8093C60031968491882324
:102D3000B1F78EEE95E0B701A6012AE030E00E94DF
:102D40009E358091C00085FFFCCF8AE08093C6004D
:102D50000E942B1547C08091680590916905A0914C
:102D60006A05B0916B0580936C0590936D05A093F7
:102D70006E05B0936F053BC0CE016AE270E00E9421
:102D8000DA570097A1F1E0E1FCE007C09091C000A4
:102D900095FFFCCF8093C600319684918823B1F7CC
:102DA000E0E9FCE007C09091C00095FFFCCF809364
:102DB000C600319684918823B1F740916C055091FB
:102DC0006D0560916E0570916F058EEE95E02AE0BD
:102DD00030E00E949E358091C00085FFFCCF8AE0E4
:102DE0008093C600109264051092630599C080918B
:102DF000DA039091DB03889D8001899D100D989DD9
:102E0000100D1124E801C452DC4FCE0167E470E0DC
:102E10000E94DA57009749F1909367058093660501
:102E20008C1B9D0B800F911F83529C4F60E070E0C4
:102E30000E94FC540E944D51DC01CB01843091056D
:102E4000A0F4872DE9EBFCE008C09091C00095FF4D
:102E5000FCCF8093C600319684918823B1F780918E
:102E6000C00085FFFCCF6092C6008091DA0390918C
:102E7000DB030196B1010E9498549093DB03809389
:102E8000DA038091D8039091D90301969093D903E6
:102E90008093D80310926405109263051EC08B3393
:102EA00011F450926505909165059923B1F4209134
:102EB000DA033091DB03289DF001299DF00D389D48
:102EC000F00D1124E40FF51FE452FC4F80834F5F97
:102ED0005F4F509364054093630580916F06909116
:102EE00070062091710630917206821B930B8F77CA
:102EF00090700097A9F08091D8039091D903843005
:102F0000910574F48EEE95E00E94E634809362059C
:102F100040916305509164058A3009F0E8CDEFCD0A
:102F2000DF91CF911F910F91FF90EF90DF90CF90A5
:102F3000BF90AF909F908F907F906F905F903F90E9
:102F40002F9008956F927F928F929F92AF92BF922F
:102F5000CF92DF92EF92FF920F931F93CF936CE289
:102F6000662E63E0762E01EC13E078E7C72E75E05D
:102F7000D72EE4EDEE2EE3E0FE2EC0E0F3018191CA
:102F80003F010E94EB14882309F10E94CF144B01EA
:102F90005C01F7018081882319F46091880501C0E4
:102FA00061E070E080E090E00E948051F8012081B3
:102FB0003181428153810E94B3539B01AC01C50111
:102FC000B4010E940550DC01CB0105C0F8018081ED
:102FD0009181A281B381F60180839183A283B3831F
:102FE000CF5F0C5F1F4F84E090E0C80ED91E08949D
:102FF000E11CF11CC43011F686E40E94EB14882316
:10300000E1F00E94CF146B017C01609396057093F0
:103010009705809398059093990520E030E040E073
:1030200050E00E94E152181644F4C0921003D0926E
:103030001103E0921203F0921303CF911F910F91AD
:10304000FF90EF90DF90CF90BF90AF909F908F90C8
:103050007F906F9008950E94A21789E40E94EB145C
:10306000882361F00E94CF14DC01CB0180939A0584
:1030700090939B05A0939C05B0939D058AE40E94C4
:10308000EB14882361F00E94CF14DC01CB01809304
:103090009E0590939F05A093A005B093A105089568
:1030A0008F929F92AF92BF92CF92DF92EF92FF9258
:1030B0000F931F93CF93DF936091FE027091FF02F5
:1030C000C8E7D5E0F4E0CF2ED12CCC0EDD1EA8E071
:1030D000AA2EB12CAC0EBD1EBCE08B2E912C8C0EFA
:1030E0009D1E882777FD8095982F0E948051209102
:1030F00010033091110340911203509113030E9469
:10310000B35320E030E040E752E40E94E55020E075
:1031100030E048EC52E40E94E5507B018C01CE0186
:10312000B601A5019401E4EBCE2EE3E0DE2E0E9471
:10313000B93F8091780590917905A0917A05B09179
:103140007B058093C1039093C203A093C303B09304
:10315000C40380917C0590917D05A0917E05B0917E
:103160007F058093C5039093C603A093C703B093D4
:10317000C8038091800590918105A0918205B0914E
:1031800083058093C9039093CA03A093CB03B093A4
:10319000CC038091840590918505A0918605B0911E
:1031A00087058093CD039093CE03A093CF03B09374
:1031B000D0030E94304FDC01CB01809370059093C7
:1031C0007105A0937205B0937305DF91CF911F91A4
:1031D0000F91FF90EF90DF90CF90BF90AF909F90B6
:1031E0008F9008954F925F926F927F92AF92BF92AD
:1031F000CF92DF92EF920F931F93CF93C82F6091DE
:103200009A0570919B0580919C0590919D05209158
:103210009E0530919F054091A0055091A1050E9407
:10322000EE522B013C016091FE027091FF0200D032
:1032300000D00DB71EB70F5F1F4F882777FD809511
:10324000982F0E94805120911003309111034091DA
:103250001203509113030E94B35320E030E040E783
:1032600052E40E94E55020E030E048EC52E40E9435
:10327000E5505B016C01F8014082518262827382E9
:10328000C4838091B403858381EC93E068E775E0A3
:103290004AE955E020E001E0A2E0EA2E0E94D236A1
:1032A0008091780590917905A0917A05B0917B0580
:1032B0008093C1039093C203A093C303B093C4034C
:1032C00080917C0590917D05A0917E05B0917F0550
:1032D0008093C5039093C603A093C703B093C8031C
:1032E0008091800590918105A0918205B091830520
:1032F0008093C9039093CA03A093CB03B093CC03EC
:103300008091840590918505A0918605B0918705EF
:103310008093CD039093CE03A093CF03B093D003BB
:103320008DB79EB706960FB6F8949EBF0FBE8DBFA1
:103330000E94304FDC01CB018093700590937105A2
:10334000A0937205B0937305CF911F910F91EF90E9
:10335000DF90CF90BF90AF907F906F905F904F9035
:103360000895F8940E949332159A179A429AA09A57
:103370008CE060E00E948E4EE0E1FCE007C090919E
:10338000C00095FFFCCF8093C600319684918823BE
:10339000B1F7E0EFFDE007C09091C00095FFFCCFD2
:1033A0008093C600319684918823B1F78091C00044
:1033B00085FFFCCF8AE08093C6000E94CC14FFCF2B
:1033C0000F931F930E94304FDC01CB014091920577
:1033D0005091930560919405709195050091700549
:1033E000109171052091720530917305801B910B2E
:1033F000A20BB30B481759076A077B0738F441152E
:1034000051056105710511F00E94B11980911503F4
:1034100090911603A0911703B09118030097A1058E
:10342000B10509F10E94304FDC01CB0140917005DC
:10343000509171056091720570917305841B950B15
:10344000A60BB70B4091150350911603609117031B
:1034500070911803481759076A077B0720F4159ADB
:10346000179A429AA09A0E94623F1F910F91089565
:10347000EF92FF920F931F93CF93DF937C018B0109
:10348000C4E0D0E0F70120813181C9010196918328
:103490008083F80161918F01C9010E944C5A2197E4
:1034A00089F784E090E0DF91CF911F910F91FF9019
:1034B000EF900895EF92FF920F931F93CF93DF93B6
:1034C0007C018B01C0E1D0E0F70120813181C9018D
:1034D000019691838083F80161918F01C9010E9457
:1034E0004C5A219789F780E190E0DF91CF911F91AD
:1034F0000F91FF90EF900895EF92FF920F931F931B
:10350000CF93DF937C018B01C4E0D0E0F7012081F1
:103510003181C901019691838083F80161918F0106
:10352000C9010E944C5A219789F784E090E0DF910D
:10353000CF911F910F91FF90EF9008950F931F93DC
:10354000CF93DF93CDB7DEB72A970FB6F894DEBFDF
:103550000FBECDBF80E390E3A0E3B0E08F839887F8
:10356000A987BA8784E690E09A838983CE01019681
:10357000BE01695F7F4F0E94381ACE01019662E951
:103580007BE00E945A1ACE01019662EA7BE00E941B
:103590005A1A02E81BE089819A819C012F5F3F4FF4
:1035A0003A832983F80161918F010E944C5AFBE014
:1035B00002391F0781F7CE0101966AE77BE00E947E
:1035C0007C1ACE01019666E77BE00E947C1ACE0150
:1035D00001966EE77BE00E947C1ACE01019666E6BA
:1035E0007BE00E947C1A02EB1BE089819A819C019E
:1035F0002F5F3F4F3A832983F80161918F010E9429
:103600004C5AFBE0063B1F0781F7CE01019662E7AB
:103610007BE00E947C1ACE0101966EE67BE00E9460
:103620007C1ACE0101966AE67BE00E947C1ACE01EC
:10363000019665E273E00E947C1ACE01019661E278
:1036400073E00E947C1ACE0101966DE173E00E9446
:103650007C1A86E590E3A5E3B0E08B839C83AD8381
:10366000BE8384E690E09A838983CE010196BE01F1
:103670006D5F7F4F0E94381AE0E5F9E007C0909136
:10368000C00095FFFCCF8093C600319684918823BB
:10369000B1F7E5EDFDE007C09091C00095FFFCCFCC
:1036A0008093C600319684918823B1F78091C00041
:1036B00085FFFCCF8AE08093C6002A960FB6F89467
:1036C000DEBF0FBECDBFDF91CF911F910F91089547
:1036D000EF92FF920F931F93CF93DF937C018B01A7
:1036E000C0E1D0E0F701808191819C012F5F3F4FC5
:1036F000318320830E94445AF80181938F012197DE
:1037000089F780E190E0DF91CF911F910F91FF90B9
:10371000EF900895EF92FF920F931F93CF93DF9353
:103720007C018B01C4E0D0E0F701808191819C0194
:103730002F5F3F4F318320830E94445AF8018193C9
:103740008F01219789F784E090E0DF91CF911F915D
:103750000F91FF90EF900895AF92BF92CF92DF92BA
:10376000EF92FF920F931F93CF93DF93CDB7DEB706
:10377000EA970FB6F894DEBF0FBECDBFD82E84E611
:1037800090E09A83898386E590E3A5E3B0E08B839C
:103790009C83AD83BE832BE0E22EF12CEC0EFD1E4C
:1037A0008E01095F1F4F89819A819C012F5F3F4FD6
:1037B0003A8329830E94445AF80181938F01EE15C0
:1037C000FF0589F7DD2009F097C0CE010396BE0101
:1037D000695F7F4F43E050E00E94E557009709F092
:1037E0008BC0CE01019662E97BE00E94681BCE018E
:1037F000019662EA7BE00E94681B02E81BE0898177
:103800009A819C012F5F3F4F3A8329830E94445A3B
:10381000F80181938F01FBE002391F0781F7CE0188
:1038200001966AE77BE00E948A1BCE01019666E75B
:103830007BE00E948A1BCE0101966EE77BE00E942E
:103840008A1BCE01019666E67BE00E948A1B02EB92
:103850001BE089819A819C012F5F3F4F3A83298326
:103860000E94445AF80181938F01FBE0063B1F0739
:1038700081F7CE01019662E77BE00E948A1BCE01B0
:1038800001966EE67BE00E948A1BCE0101966AE6F5
:103890007BE00E948A1BCE01019665E273E00E94E4
:1038A0008A1BCE01019661E273E00E948A1BCE0161
:1038B00001966DE173E00E948A1BE0E5F9E007C024
:1038C0009091C00095FFFCCF8093C6003196849103
:1038D0008823B1F7E8E6FAE007C09091C00095FFB1
:1038E000FCCF8093C600319684918823B1F78091F4
:1038F000C00085FFFCCFCEC0DE019B96E1E3F2E085
:1039000080E101900D928150E1F7DE015B96E1E4E8
:10391000F2E080E101900D928150E1F7DE011B960B
:10392000E1E5F2E080E101900D928150E1F7BBE228
:10393000AB2EB12CAC0EBD1E42E95BE0BE01655E54
:103940007F4F02EA1BE08BE0E82EF12CEC0EFD1E0F
:1039500092E8C92E9BE0D92E24E030E0F501819158
:103960009191A191B1915F01FA0181939193A193FA
:10397000B193AF01FB0181919191A191B191BF01EF
:10398000F80181939193A193B1938F01F7018191F4
:103990009191A191B1917F01F60181939193A193AE
:1039A000B1936F0121503040C9F680E090E8ABE35D
:1039B000B5E480937A0B90937B0BA0937C0BB09330
:1039C0007D0B8093760B9093770BA093780BB0933D
:1039D000790B80E090E0A0E0B0E080937E0B9093C4
:1039E0007F0BA093800BB093810B40E25EE460E01C
:1039F00070E04093B20B5093B30B6093B40B709391
:103A0000B50B8093660B9093670BA093680BB093F4
:103A1000690B80E090E0A0EAB1E48093720B909390
:103A2000730BA093740BB093750B8DEC9CECACEC0A
:103A3000BEE380936E0B90936F0BA093700BB093CB
:103A4000710B80E090E0A0EAB0E480936A0B909361
:103A50006B0BA0936C0BB0936D0BE0E5F9E007C026
:103A60009091C00095FFFCCF8093C6003196849161
:103A70008823B1F7E9E1F2E006C09091C00095FF1C
:103A8000FCCF8093C60081918823B9F78091C00054
:103A900085FFFCCF8AE08093C6000E94D510EA968D
:103AA0000FB6F894DEBF0FBECDBFDF91CF911F914F
:103AB0000F91FF90EF90DF90CF90BF90AF9008955F
:103AC0002F923F924F925F926F927F928F929F922E
:103AD000AF92BF92CF92DF92EF92FF920F931F931C
:103AE000CF93DF93CDB7DEB7A2970FB6F894DEBFC2
:103AF0000FBECDBF87E40E94EB14882309F4C7C52D
:103B00000E94CF140E944D5164307105A9F16530B7
:103B1000710554F46230710521F1633071052CF5A3
:103B200077FF19C00C944F2D6A35710509F445C50E
:103B30006B35710534F46C31710511F00C944F2D17
:103B40005FC06B35710509F43CC56C35710511F02A
:103B50000C944F2D3BC50E94A2170E9450180C9444
:103B6000742D0E942B1881E003C00E942B1880E066
:103B70000E94F2180C94742D80E50E94EB148823A7
:103B800039F00E94CF140E9452516B017C0103C096
:103B9000CC24DD24760183E50E94EB14882361F0B8
:103BA0000E94CF1420E030E04AE754E40E94B3536F
:103BB0000E9452516B017C010E945E100E94304FA6
:103BC0004B015C018C0C9D1CAE1CBF1C0E94304F35
:103BD000DC01CB018093700590937105A093720571
:103BE000B093730502C00E9411300E94304FDC0177
:103BF000CB0188159905AA05BB05A8F30C944F2D98
:103C00008091100390911103A0911203B0911303BE
:103C10008093740590937505A0937605B09377050E
:103C20008091FE029091FF029093D3038093D20380
:103C300084E690E09093FF028093FE0281E00E9470
:103C400025098091C1039091C203A091C303B09153
:103C5000C4038093780590937905A0937A05B09377
:103C60007B058091C5039091C603A091C703B091D5
:103C7000C80380937C0590937D05A0937E05B09347
:103C80007F058091C9039091CA03A091CB03B091A5
:103C9000CC038093800590938105A0938205B09317
:103CA00083058091CD039091CE03A091CF03B09175
:103CB000D0038093840590938505A0938605B093E7
:103CC000870580E090E0A0E0B0E08093100390933F
:103CD0001103A0931203B093130388E50E94EB1421
:103CE000882361F489E50E94EB14882339F48AE57E
:103CF0000E94EB14882311F481E001C080E08093DE
:103D0000140388E50E94EB14882309F4E8C089E5D0
:103D10000E94EB14882309F4E2C080E090E0A0E068
:103D2000B0E08093C1039093C203A093C303B09308
:103D3000C4038093C5039093C603A093C703B093B5
:103D4000C80381EC93E065EC73E049EC53E02DECA3
:103D500033E00E94E54A80E090ECA9E9B3EC80935F
:103D6000780590937905A0937A05B0937B058093AD
:103D70007C0590937D05A0937E05B0937F052091EF
:103D800000033091010340910203509103032093FB
:103D90001003309311034093120350931303C09008
:103DA0000403D0900503E0900603F0900703C701D9
:103DB000B6010E94DE5087FF08C0C0921003D09267
:103DC0001103E0921203F0921303609110037091BB
:103DD0001103809112039091130320E030E040E73B
:103DE00052E40E94E5507B018C0188E795E06CE786
:103DF00075E040E855E024E835E0F4EBCF2EF3E041
:103E0000DF2E0E94B93F0E945E100F2EF0E08F2E31
:103E1000F0E09F2EF0E0AF2EF0E0BF2EF02D80926C
:103E2000C1039092C203A092C303B092C4038092D4
:103E3000C5039092C603A092C703B092C80381EC59
:103E400093E065EC73E049EC53E02DEC33E00E9425
:103E5000E54A8091C1039091C203A091C303B09140
:103E6000C4038093780590937905A0937A05B09365
:103E70007B058091C5039091C603A091C703B091C3
:103E8000C80380937C0590937D05A0937E05B09335
:103E90007F0560911003709111038091120390913E
:103EA000130320E030E040E752E40E94E5507B013C
:103EB0008C0188E795E06CE775E040E855E024E880
:103EC00035E00E94B93F8092100390921103A092B6
:103ED0001203B09213030E945E100E941E0980918B
:103EE0001403882331F488E50E94EB14882309F435
:103EF000E7C00F2EF0E08F2EF0E09F2EF0E0AF2E07
:103F0000F0E0BF2EF02D8092C1039092C203A092E8
:103F1000C303B092C40381EC93E065EC73E049EC19
:103F200053E02DEC33E00E94E54A80E090ECA9E9F3
:103F3000B3EC8093780590937905A0937A05B093BC
:103F40007B056091000370910103809102039091C1
:103F500003036093100370931103809312039093F3
:103F6000130320E030E040E752E40E94E5507B017B
:103F70008C0188E795E06CE775E040E855E024E8BF
:103F800035E0E4EBCE2EE3E0DE2E0E94B93F0E9446
:103F90005E108092C1039092C203A092C303B092BC
:103FA000C40381EC93E065EC73E049EC53E02DEC45
:103FB00033E00E94E54A80E090E0A0EAB0E480931C
:103FC000780590937905A0937A05B0937B0560916D
:103FD000100370911103809112039091130320E05C
:103FE00030E040E752E40E94E5507B018C0188E715
:103FF00095E06CE775E040E855E024E835E00E9484
:10400000B93F0E945E1080E090E0A0E2B1EC8093A6
:10401000780590937905A0937A05B0937B0560911C
:10402000000370910103809102039091030320E04B
:1040300030E040E05FE30E94B3539B01F82FE92F8B
:10404000462F532F682F792F40931003509311035D
:104050006093120370931303822F932FAF2FBE2F01
:10406000BC01CD0120E030E040E752E40E94E55081
:104070007B018C0188E795E06CE775E040E855E04E
:1040800024E835E00E94B93F0E945E108092C1038F
:104090009092C203A092C303B092C40380927805A9
:1040A00090927905A0927A05B0927B0580921003D8
:1040B00090921103A0921203B09213030E941E0962
:1040C00080911403882331F489E50E94EB1488233E
:1040D00009F4E7C00F2EF0E08F2EF0E09F2EF0E005
:1040E000AF2EF0E0BF2EF02D8092C5039092C60354
:1040F000A092C703B092C80381EC93E065EC73E033
:1041000049EC53E02DEC33E00E94E54A80E090EC6E
:10411000A9E9B3EC80937C0590937D05A0937E057F
:10412000B0937F05609104037091050380910603AD
:10413000909107036093100370931103809312030F
:104140009093130320E030E040E752E40E94E550F2
:104150007B018C0188E795E06CE775E040E855E06D
:1041600024E835E0F4EBCF2EF3E0DF2E0E94B93FD8
:104170000E945E108092C5039092C603A092C7036E
:10418000B092C80381EC93E065EC73E049EC53E036
:104190002DEC33E00E94E54A80E090E0A0EAB0E434
:1041A00080937C0590937D05A0937E05B0937F0559
:1041B0006091100370911103809112039091130389
:1041C00020E030E040E752E40E94E5507B018C01A2
:1041D00088E795E06CE775E040E855E024E835E0D5
:1041E0000E94B93F0E945E1080E090E0A0E2B1EC36
:1041F00080937C0590937D05A0937E05B0937F0509
:104200006091040370910503809106039091070368
:1042100020E030E040E05FE30E94B3539B01F82FC1
:10422000E92F462F532F682F792F40931003509377
:1042300011036093120370931303822F932FAF2FF8
:10424000BE2FBC01CD0120E030E040E752E40E94E7
:10425000E5507B018C0188E795E06CE775E040E86C
:1042600055E024E835E00E94B93F0E945E1080923C
:10427000C5039092C603A092C703B092C803809270
:104280007C0590927D05A0927E05B0927F0580927C
:10429000100390921103A0921203B09213030E9494
:1042A0001E0980911403882331F48AE50E94EB14DF
:1042B000882309F4E7C00F2EF0E08F2EF0E09F2E48
:1042C000F0E0AF2EF0E0BF2EF02D8092C903909267
:1042D000CA03A092CB03B092CC0381EC93E065ECCF
:1042E00073E049EC53E02DEC33E00E94E54A80E0B6
:1042F00090E0A6E9B3EC8093800590938105A093AC
:104300008205B09383056091080370910903809141
:104310000A0390910B036093100370931103809331
:1043200012039093130320E030E040E752E40E9430
:10433000E5507B018C0188E795E06CE775E040E88B
:1043400055E024E835E0E4EBCE2EE3E0DE2E0E94DB
:10435000B93F0E945E108092C9039092CA03A09256
:10436000CB03B092CC0381EC93E065EC73E049ECB5
:1043700053E02DEC33E00E94E54A80E090E0A0E8B5
:10438000BFE38093800590938105A0938205B0934D
:104390008305609110037091110380911203909135
:1043A000130320E030E040E752E40E94E5507B0137
:1043B0008C0188E795E06CE775E040E855E024E87B
:1043C00035E00E94B93F0E945E1080E090E0A0E0DE
:1043D000B0EC8093800590938105A0938205B09303
:1043E0008305609108037091090380910A039091FD
:1043F0000B0320E030E040E05FE30E94B3539B01F9
:10440000F82FE92F462F532F682F792F4093100351
:10441000509311036093120370931303822F932F11
:10442000AF2FBE2FBC01CD0120E030E040E752E4C9
:104430000E94E5507B018C0188E795E06CE775E010
:1044400040E855E024E835E00E94B93F0E945E1044
:104450008092C9039092CA03A092CB03B092CC037E
:104460008092800590928105A0928205B09283058A
:104470008092100390921103A0921203B092130342
:104480000E941E0988E50E94EB148823F1F00E9427
:10449000DF14DC01CB010097A105B105B1F00E944A
:1044A000CF142091B5033091B6034091B7035091DA
:1044B000B8030E940550DC01CB018093C1039093A7
:1044C000C203A093C303B093C40389E50E94EB1415
:1044D0008823F1F00E94DF14DC01CB010097A105D5
:1044E000B105B1F00E94CF142091B9033091BA0305
:1044F0004091BB035091BC030E940550DC01CB01ED
:104500008093C5039093C603A093C703B093C803D9
:104510008AE50E94EB148823F1F00E94DF14DC018D
:10452000CB010097A105B105B1F00E94CF142091F5
:10453000BD033091BE034091BF035091C0030E9460
:104540000550DC01CB018093C9039093CA03A0936B
:10455000CB03B093CC0381EC93E065EC73E049ECC2
:1045600053E02DEC33E00E94E54A80917405909170
:104570007505A0917605B09177058093100390930F
:104580001103A0931203B09313038091D20390916F
:10459000D3039093FF028093FE020E94304FDC0110
:1045A000CB018093700590937105A0937205B09331
:1045B00073050E941E090C944F2D109288050C94CF
:1045C0004F2D81E0809388050C944F2D85E40E9447
:1045D000EB14882311F40E945E103CE2832E33E03A
:1045E000932E45EBC42E43E0D42E51ECE52E53E040
:1045F000F52E00E0F40181914F010E94EB14882315
:10460000D1F10E94CF14F601208131814281538182
:104610000E940550DC01CB01F70180839183A283C6
:10462000B383033071F40E94CF14DC01CB01F70196
:1046300080839183A283B3838DEC93E00E94954B9A
:104640001AC00E94CF14F60120813181428153812A
:104650000E940550DC01CB01F70180839183A28386
:10466000B38381EC93E065EC73E049EC53E02DEC0F
:1046700033E00E94E54A0F5F24E030E0C20ED31E13
:10468000E20EF31E043009F0B5CF0C944F2D8DE4EB
:104690000E94EB14882311F40C94A12C0E94CF14D7
:1046A0000E944D516337710509F484C56437710563
:1046B0000CF05AC06435710509F4FBC46535710509
:1046C00064F56A32710509F434C16B32710574F412
:1046D0006231710509F4EDC46F31710509F4BAC096
:1046E0006131710511F00C944F2DAEC0613571052B
:1046F00009F4D3C46235710534F46035710511F0E5
:104700000C944F2DC8C46235710509F4CBC46335D0
:10471000710511F00C944F2DC8C46936710509F468
:10472000C7C16A36710574F46C35710509F424C586
:104730006836710509F445C16535710511F00C94B1
:104740004F2D02C56B36710509F4A2C46B36710595
:104750000CF476C46D36710509F43FC262377105F9
:1047600011F00C944F2D34C56C3D710511F40C946F
:10477000862B6D3D710564F5693C710509F4BEC673
:104780006A3C710574F46C38710509F47CC16E3BA8
:10479000710509F4B6C36737710511F00C944F2DFC
:1047A000F3C56C3C710509F405C76D3C710534F423
:1047B0006B3C710511F00C944F2DDEC66D3C7105FC
:1047C00009F41CC76E3C710511F00C944F2D80C785
:1047D00031E06039730711F40C94922C81E0613957
:1047E000780794F491E06D32790711F40C94AB2BB7
:1047F000E1E06E327E0711F40C948E2C6D3D710554
:1048000011F00C944F2D96C7F1E0653F7F0711F42E
:104810000C94982C21E0663F720744F431E0643F29
:10482000730711F00C944F2D0C94952C81E0663F8A
:10483000780711F40C949A2C91E0673F790711F0F6
:104840000C944F2D0C949E2C159817984298A09874
:104850000C944F2D0E94304FDC01CB0180938905D1
:1048600090938A05A0938B05B0938C0540918D059C
:1048700050918E0560918F0570919005841B950B6A
:10488000A60BB70BBC01CD0128EE33E040E050E0B1
:104890000E94AB54EDB7FEB738970FB6F894FEBF41
:1048A0000FBEEDBF0DB71EB70F5F1F4FCE010196B4
:1048B0009283818387E692E0F80193838283CA0121
:1048C000B9012CE330E040E050E00E94AB54DC0141
:1048D000CB01F80135832483978386830E940D588A
:1048E000E0E5F9E084912DB73EB7285F3F4F0FB662
:1048F000F8943EBF0FBE2DBF08C09091C00095FF39
:10490000FCCF8093C600319684918823B1F7FE01D5
:10491000319606C09091C00095FFFCCF8093C600F1
:1049200081918823B9F78091C00085FFFCCF0C945A
:104930004C2D83E50E94EB14882311F40C944F2D29
:104940000E94CF146B017C0180E50E94EB14882348
:1049500011F40C944F2DC701B6010E944D51DC019A
:10496000CB017C0197FF02C00C944F2D8F3F910526
:1049700019F014F00C944F2D0E94CF140E944D5149
:104980008B019C01E0E3F3E020E08191919180179D
:10499000910711F40C944F2D2F5F2A33B1F717FFB5
:1049A00002C00C944F2D802F61E00E948E4E802F0C
:1049B0006E2D0E94AF4E802FB7010E943E4D0C9489
:1049C0004F2D8091B4038093910584E50E94EB14F0
:1049D000882379F10E94CF140E945251609391056F
:1049E000662339F1E0E5F9E007C09091C00095FF3A
:1049F000FCCF8093C600319684918823B1F7E6E717
:104A0000F2E006C09091C00095FFFCCF8093C600F5
:104A100081918823B9F78EEE95E06091910540E091
:104A200050E00E9496358091C00085FFFCCF0C9429
:104A30004C2D83E50E94EB14882309F10E94CF14CA
:104A40006B017C0100919105802E99240E944D51AB
:104A5000DC01CB01602F0E94752FF401EE0FFF1FC8
:104A6000E055FA4F91838083F401EE0FFF1FEE0FA4
:104A7000FF1FEA55FA4FC082D182E282F3820E9480
:104A800092320C944F2D83E50E94EB14882311F48D
:104A90000C944F2D0E94CF140E944D51DC01CB018C
:104AA0000E94BD2F9093AF058093AE050C944F2DBF
:104AB0008091B4038093910584E50E94EB148823D0
:104AC00079F10E94CF140E945251609391056623A0
:104AD00039F1E0E5F9E007C09091C00095FFFCCF07
:104AE0008093C600319684918823B1F7EDE8F2E017
:104AF00006C09091C00095FFFCCF8093C6008191C5
:104B00008823B9F78EEE95E06091910540E050E082
:104B10000E9496358091C00085FFFCCF0C944C2DEF
:104B2000ECEBFCE007C09091C00095FFFCCF8093B8
:104B3000C600319684918823B1F760919105E62FE4
:104B4000F0E0EE0FFF1FE455FA4F808191810E9443
:104B5000C02FAB01BC018EEE95E022E030E00E9458
:104B6000CF36E2ECFCE007C09091C00095FFFCCF8F
:104B70008093C600319684918823B1F78091AA056D
:104B80009091AB050E943032AB01BC018EEE95E0F6
:104B900022E030E00E94CF36E6ECFCE007C09091C6
:104BA000C00095FFFCCF8093C60031968491882386
:104BB000B1F78091910590E00E946F2FBC018EEEBD
:104BC00095E04AE050E00E94D3358091C00085FF17
:104BD000FCCF8AE08093C60087C78091B40380939E
:104BE000910584E50E94EB14882371F10E94CF1493
:104BF0000E94525160939105662331F1E0E5F9E09E
:104C000007C09091C00095FFFCCF8093C6003196FD
:104C100084918823B1F7E4EAF2E006C09091C000E5
:104C200095FFFCCF8093C60081918823B9F78EEE63
:104C300095E06091910540E050E00E9496358091AA
:104C4000C00085FFFCCF28C783E50E94EB148823B2
:104C500009F10E94CF146B017C0100919105802E17
:104C600099240E944D51DC01CB01602F0E94752FC9
:104C7000F401EE0FFF1FE055FA4F91838083F4019A
:104C8000EE0FFF1FEE0FFF1FEA55FA4FC082D182D1
:104C9000E282F3820E9492320E94304F2B013C014B
:104CA0008091910590E0880F991FFC01E055FA4F23
:104CB0002081318138A32F8F84559A4FFC010190B8
:104CC000F081E02DFAA3E9A388248A94982C54015A
:104CD000EAECFCE03490EDECFCE02490E1EDFCE04B
:104CE00004911AE0FCC0832DEAECFCE008C090912E
:104CF000C00095FFFCCF8093C60031968491882335
:104D0000B1F760919105E62FF0E0EE0FFF1FE4553B
:104D1000FA4F808191810E94C02FAB01BC018EEEC1
:104D200095E022E030E00E94CF36822DEDECFCE0F1
:104D300008C09091C00095FFFCCF8093C6003196CB
:104D400084918823B1F7609191058EEE95E070E033
:104D50004AE050E00E94D335802FE1EDFCE008C02E
:104D60009091C00095FFFCCF8093C600319684914E
:104D70008823B1F7B7FE03C0EBEBF2E029C00E9435
:104D8000304FAB01BC01D501C401805D9A48AF4FE3
:104D9000BF4F841B950BA60BB70BBC01CD0128EEB2
:104DA00033E040E050E00E94AB548EEE95E0BA0153
:104DB000A9012AE030E00E9489358091C00085FF7A
:104DC000FCCF0DC09091C00095FFFCCF8093C60032
:104DD00081918823B9F78091C00085FFFCCF1093A3
:104DE000C6000E94304F2B013C010E941130FFEFA2
:104DF0008F16FFEF9F06FFEFAF06FFEFBF0619F517
:104E0000A09191052F8D38A189A19AA1B0E0AA0F98
:104E1000BB1FFD01E055FA4FA455BA4F8217930707
:104E20004CF4808191812D913C911197281739077D
:104E3000F4F541C0808191812D913C9111978217A9
:104E40009307ACF538C0B7FC36C060919105E62FEA
:104E5000F0E0EE0FFF1FE455FA4F808191810E9430
:104E6000C02F6B017C0160919105E62FF0E0EE0F01
:104E7000FF1FE055FA4F808191810E94C02F9B0156
:104E8000AC01C701B6010E9404500E944D51AB0114
:104E9000BC0177FF07C070956095509541955F4FB5
:104EA0006F4F7F4F443051056105710524F00E941A
:104EB000304F4B015C019FEF89169FEF99069FEFE2
:104EC000A9069FEFB90659F0B7FCECC50E94304F18
:104ED00068197909E5E760337E0708F0E3C50E94A9
:104EE000304FDC01CB0184199509A609B709893E29
:104EF000F3E09F07F0E0AF07F0E0BF0708F0F3CE64
:104F000074CF83E50E94EB14882361F00E94CF14D4
:104F10000E944D51DC01CB010E94BD2F9093AF0543
:104F20008093AE050E94304F6B017C01E5EDFCE003
:104F3000B490E8EDFCE08490ECEDFCE004911AE024
:104F400072C00E94304FDC01CB018C199D09AE0963
:104F5000BF09893E23E0920720E0A20720E0B207C4
:104F600008F45FC06091B403E62FF0E0EE0FFF1F7E
:104F7000E455FA4F808191810E94C02FAB01BC01A2
:104F80008B2DE5EDFCE008C09091C00095FFFCCFB3
:104F90008093C600319684918823B1F78EEE95E018
:104FA00022E030E00E94CF36882DE8EDFCE008C01A
:104FB0009091C00095FFFCCF8093C60031968491FC
:104FC0008823B1F76091B4038EEE95E070E04AE07B
:104FD00050E00E94D335802FECEDFCE008C09091AA
:104FE000C00095FFFCCF8093C60031968491882342
:104FF000B1F78091AA059091AB050E943032AB01C8
:10500000BC018EEE95E022E030E00E94CF36809128
:10501000C00085FFFCCF1093C6000E94304F6B018B
:105020007C010E9411302091AE053091AF05809136
:10503000AA059091AB05821793070CF482CF3EC569
:1050400083E50E94EB148823F9F00E94CF1420E03E
:1050500030E040E050E00E94DE5087FD0FC00E942B
:10506000CF1420E030E04FE753E40E94E1521816DD
:105070003CF00E94CF140E94525103C060E001C076
:105080006FEF6093B3030BC58FEF8093B30307C536
:105090001092B30304C5269A02C50E945E100E94B6
:1050A000CC14FDC41092D703FAC481E08093D703D7
:1050B000F6C483E50E94EB148823A9F00E94CF1464
:1050C00020E030E04AE754E40E94B3530E9452517A
:1050D000DC01CB018093150390931603A093170373
:1050E000B0931803DCC488E50E94EB14882309F010
:1050F000F2C489E50E94EB14882309F0ECC48AE528
:105100000E94EB14882309F0E6C485E40E94EB14A6
:10511000882309F0E0C40E945E10A09A0E94CE107D
:10512000BEC4159A89E50E94EB148111179A8AE58D
:105130000E94EB148111429A85E40E94EB148823AB
:1051400009F4ADC4A09AABC483E50E94EB140E949D
:10515000CF1420E030E04AE754E40E94B3530E94A9
:105160005251DC01CB018093920590939305A0935B
:105170009405B093950593C44CE2C42E43E0D42E1D
:1051800002E91BE0EE24F60181916F010E94EB140D
:10519000882349F00E94CF14DC01CB01F801808301
:1051A0009183A283B383E3940C5F1F4FF4E0EF1667
:1051B00051F775C4E0EEFCE007C09091C00095FF88
:1051C000FCCF8093C600319684918823B1F767C4E1
:1051D000EBE7FDE007C09091C00095FFFCCF809306
:1051E000C600319684918823B1F74091C103509154
:1051F000C2036091C3037091C4038EEE95E022E078
:1052000030E00E94CF36EEE7FDE007C09091C0008D
:1052100095FFFCCF8093C600319684918823B1F727
:105220004091C5035091C6036091C7037091C803B4
:105230008EEE95E022E030E00E94CF36E1E8FDE01E
:1052400007C09091C00095FFFCCF8093C6003196B7
:1052500084918823B1F74091C9035091CA036091AA
:10526000CB037091CC038EEE95E022E030E00E94FB
:10527000CF36E4E8FDE007C09091C00095FFFCCF79
:105280008093C600319684918823B1F74091CD0375
:105290005091CE036091CF037091D0038EEE95E0D4
:1052A00022E030E00E94CF36E7E8FDE007C09091B1
:1052B000C00095FFFCCF8093C6003196849188236F
:1052C000B1F70E94B8100E9480512091920B30914A
:1052D000930B4091940B5091950B0E94E550AB01BC
:1052E000BC018EEE95E022E030E00E94CF36E1E98D
:1052F000FDE007C09091C00095FFFCCF8093C600F1
:10530000319684918823B1F781E00E94B8100E9401
:1053100080512091960B3091970B4091980B5091B2
:10532000990B0E94E550AB01BC018EEE95E022E0A6
:1053300030E00E94CF36E4E9FDE007C09091C00064
:1053400095FFFCCF8093C600319684918823B1F7F6
:1053500082E00E94B8100E94805120919A0B3091F7
:105360009B0B40919C0B50919D0B0E94E550AB0113
:10537000BC018EEE95E022E030E00E94CF368091B5
:10538000C00085FFFCCF88C3E7E9FDE007C090912E
:10539000C00095FFFCCF8093C6003196849188238E
:1053A000B1F780B180FD03C0E1E6F2E009C0E4E6B8
:1053B000F2E006C09091C00095FFFCCF8093C6003C
:1053C00081918823B9F7EEE9FDE007C09091C00014
:1053D00095FFFCCF8093C600319684918823B1F766
:1053E000029903C0E1E6F2E009C0E4E6F2E006C09B
:1053F0009091C00095FFFCCF8093C60081918823D7
:10540000B9F7E5EAFDE007C09091C00095FFFCCF39
:105410008093C600319684918823B1F7049903C024
:10542000E1E6F2E009C0E4E6F2E006C09091C000D7
:1054300095FFFCCF8093C60081918823B9F7ECEAF1
:10544000FDE007C09091C00095FFFCCF8093C6009F
:10545000319684918823B1F7069903C0E1E6F2E022
:1054600009C0E4E6F2E006C09091C00095FFFCCFD1
:105470008093C60081918823B9F7E3EBFDE007C074
:105480009091C00095FFFCCF8093C6003196849127
:105490008823B1F7379903C0E1E6F2E009C0E4E6FA
:1054A000F2E006C09091C00095FFFCCF8093C6004B
:1054B00081918823B9F7EAEBFDE007C09091C00025
:1054C00095FFFCCF8093C600319684918823B1F775
:1054D000359903C0E1E6F2E009C0E4E6F2E006C077
:1054E0009091C00095FFFCCF8093C60081918823E6
:1054F000B9F78091C00085FFFCCFCEC23CE2C32E3D
:1055000033E0D32E00E010E0F60181916F010E949C
:10551000EB14882359F10E94CF14E2E8EE2EEBE061
:10552000FE2EE00EF11E0E945251DC01CB01F7016C
:1055300080839183A283B3830E94CF1426E5E22E59
:105540002BE0F22EE00EF11EF801EE56F44F208112
:105550003181428153810E94B3530E945251DC0138
:10556000CB01F70180839183A283B3830C5F1F4F2C
:105570000031110549F693C25CE2C52E53E0D52EE9
:1055800002EA1BE064E0E62EF60181916F010E94C1
:10559000EB14882349F00E94CF14DC01CB01F80101
:1055A00080839183A283B383EA940C5F1F4FEE2024
:1055B00059F775C283E50E94EB14882361F00E94BD
:1055C000CF14DC01CB0180937A0B90937B0BA093DB
:1055D0007C0BB0937D0B84E50E94EB14882309F4C7
:1055E0005EC20E94CF14DC01CB018093760B9093B6
:1055F000770BA093780BB093790B51C283E50E948F
:10560000EB14882361F00E94CF14DC01CB0180935E
:105610007E0B90937F0BA093800BB093810B84E55E
:105620000E94EB14882361F00E94CF14DC01CB01AF
:105630008093660B9093670BA093680BB093690BF4
:1056400082E40E94EB14882371F00E94CF140E9420
:105650005251DC01CB018093B20B9093B30BA0931A
:10566000B40BB093B50B88E50E94EB14882361F06E
:105670000E94CF14DC01CB018093720B9093730BCB
:10568000A093740BB093750B8AE50E94EB148823EA
:1056900061F00E94CF14DC01CB0180936E0B9093DC
:1056A0006F0BA093700BB093710B85E40E94EB1409
:1056B000882309F4F4C10E94CF14DC01CB0180934C
:1056C0006A0B90936B0BA0936C0BB0936D0BE7C1BF
:1056D0003CE2C32E33E0D32E05EB13E043E0E42E8F
:1056E000F60181916F010E94EB14882349F00E941A
:1056F000CF14DC01CB01F80180839183A283B383B3
:10570000EA940C5F1F4FEE2059F7C9C183E50E9450
:10571000EB14882309F4C3C10E94CF140E944D5199
:10572000DC01CB019093FF028093FE0281E0809325
:10573000D103B5C183E50E94EB14882309F4AFC1FE
:105740000E94CF140E944D51DC01CB019093FD02C9
:105750008093FC02A4C180E50E94EB14882361F0D1
:105760000E94CF14DC01CB01809325039093260384
:10577000A0932703B093280389E40E94EB148823A5
:1057800091F00E94CF142FE632E143E05EE30E94E5
:10579000B353DC01CB018093210390932203A093A8
:1057A0002303B093240384E40E94EB14882391F034
:1057B0000E94CF142FE632E143E05EE30E94E55001
:1057C000DC01CB0180931D0390931E03A0931F0364
:1057D000B093200383E40E94EB14882361F00E94BD
:1057E000CF14DC01CB018093190390931A03A0938B
:1057F0001B03B0931C030E94562FEDEBF2E006C092
:105800009091C00095FFFCCF8093C60081918823C2
:10581000B9F7E0ECF2E006C09091C00095FFFCCF34
:105820008093C60081918823B9F740912503509158
:10583000260360912703709128038EEE95E022E005
:1058400030E00E94CF36E4ECF2E006C09091C00058
:1058500095FFFCCF8093C60081918823B9F76091B2
:1058600021037091220380912303909124032FE65A
:1058700032E143E05EE30E94E550AB01BC018EEEF5
:1058800095E022E030E00E94CF36E8ECF2E006C07E
:105890009091C00095FFFCCF8093C6008191882332
:1058A000B9F760911D0370911E0380911F039091C1
:1058B00020032FE632E143E05EE30E94B353AB01E5
:1058C000BC018EEE95E022E030E00E94CF36ECEC99
:1058D000F2E006C09091C00095FFFCCF8093C60017
:1058E00081918823B9F76091190370911A0380910F
:1058F0001B0390911C032FE632E143E05EE30E941C
:10590000B353AB01BC018EEE95E022E030E00E9483
:10591000CF368091C00085FFFCCFBEC081E00E94E1
:10592000B34BBDC00E945E10BAC00E949E1AB7C0A1
:1059300080E001C081E00E94AC1BB1C00E94D51084
:10594000AEC084E50E94EB14882309F461C00E9474
:10595000CF140E94525160939105E0E5F9E066236F
:1059600081F107C09091C00095FFFCCF8093C600E5
:10597000319684918823B1F7E0EDF2E006C0909172
:10598000C00095FFFCCF8093C60081918823B9F7B2
:105990008EEE95E06091910540E050E00E949635D2
:1059A000E2EDF2E006C09091C00095FFFCCF80933D
:1059B000C60081918823B9F78091C00085FFFCCF94
:1059C0006BC01092B40307C09091C00095FFFCCF4C
:1059D0008093C600319684918823B1F7E3EEF2E01C
:1059E00006C09091C00095FFFCCF8093C6008191C6
:1059F0008823B9F76091B4038EEE95E070E04AE039
:105A000050E00E94D3358091C00085FFFCCF44C098
:105A1000E0E5F9E007C09091C00095FFFCCF8093CE
:105A2000C600319684918823B1F7E1ECFDE007C010
:105A30009091C00095FFFCCF8093C6003196849171
:105A40008823B1F7209160053091610580E690E0F0
:105A5000289FF001299FF00D389FF00D1124E4528A
:105A6000FC4F06C09091C00095FFFCCF8093C6000C
:105A700081918823B9F7E3EDFDE007C09091C00064
:105A800095FFFCCF8093C600319684918823B1F7AF
:105A90008091C00085FFFCCF8AE08093C6000E9401
:105AA0000A1522C00E94304FDC01CB0180938D0586
:105AB00090938E05A0938F05B09390050E94304F70
:105AC000DC01CB018093700590937105A093720562
:105AD000B0937305E4CF0E945E1088E50E94EB143A
:105AE000882309F01ECB1ECBA2960FB6F894DEBF1A
:105AF0000FBECDBFDF91CF911F910F91FF90EF901F
:105B0000DF90CF90BF90AF909F908F907F906F90DD
:105B10005F904F903F902F9008958091D80390917F
:105B2000D9038330910514F40E9458158091D8034D
:105B30009091D9030097C1F00E94601D8091D80315
:105B40009091D90301979093D9038093D8038091C2
:105B5000600590916105019664E070E00E949854A0
:105B600090936105809360050E94113081E00E944E
:105B7000E0190E94620808958F929F92AF92BF929F
:105B8000CF92DF92EF92FF920F931F93CF930E94D9
:105B9000C9148EEE95E040E950ED63E070E00E949C
:105BA000A834E3E6F9E007C09091C00095FFFCCF70
:105BB0008093C600319684918823B1F78091C0000C
:105BC00085FFFCCF8AE08093C60080E599E0FC0168
:105BD00007C03091C00035FFFCCF2093C60031963E
:105BE00024912223B1F724B720FF14C0E9E6F9E09D
:105BF00007C04091C00045FFFCCF3093C6003196EE
:105C000034913323B1F73091C00035FFFCCF3AE037
:105C10003093C60021FF14C0E1E7F9E007C04091CE
:105C2000C00045FFFCCF3093C6003196349133233A
:105C3000B1F73091C00035FFFCCF3AE03093C60099
:105C400022FF14C0E1E8F9E007C04091C00045FF21
:105C5000FCCF3093C600319634913323B1F73091A5
:105C6000C00035FFFCCF3AE03093C60023FF14C0DC
:105C7000E2E9F9E007C04091C00045FFFCCF309356
:105C8000C600319634913323B1F73091C00035FF0F
:105C9000FCCF3AE03093C60025FF14C0E2EAF9E0F9
:105CA00007C03091C00035FFFCCF2093C60031966D
:105CB00024912223B1F72091C00025FFFCCF2AE0D8
:105CC0002093C60014BEE2EBF9E007C03091C0009B
:105CD00035FFFCCF2093C600319624912223B1F7E3
:105CE000EBEBF9E007C03091C00035FFFCCF20930B
:105CF000C600319624912223B1F72091C00025FFE0
:105D0000FCCF2AE02093C600FC012491E0E5F9E0F5
:105D100008C03091C00035FFFCCF2093C6003196FB
:105D200024912223B1F7E5ECF9E007C03091C000DF
:105D300035FFFCCF2093C600319624912223B1F782
:105D4000E5EDF9E007C03091C00035FFFCCF2093AE
:105D5000C600319624912223B1F7E6E2FAE007C0AB
:105D60003091C00035FFFCCF2093C60031962491BE
:105D70002223B1F7E2E3FAE007C03091C00035FF1B
:105D8000FCCF2093C600319624912223B1F72091B5
:105D9000C00025FFFCCF2AE02093C600FC018491BF
:105DA000E0E5F9E008C09091C00095FFFCCF80933A
:105DB000C600319684918823B1F7E2E4FAE007C087
:105DC0009091C00095FFFCCF8093C60031968491DE
:105DD0008823B1F70E94AC14BC018EEE95E04AE036
:105DE00050E00E94D335E1E5FAE007C09091C00091
:105DF00095FFFCCF8093C600319684918823B1F73C
:105E00008EEE95E060ED74E04AE050E00E94D335FC
:105E10008091C00085FFFCCF8AE08093C60010927D
:105E20005C0510925D0510925E0510925F0580E0A2
:105E30000E94AC1B02E81BE0A2E9AA2EABE0BA2E3E
:105E4000B6E58B2EBBE09B2EC0E0F801619171910D
:105E5000819191918F01F501C190D190E190F190E4
:105E60005F010E947E51A70196010E94B3530E94D8
:105E70005251DC01CB01F40181939193A193B19331
:105E80004F01CF5FC43009F70E9435320E942A3F8C
:105E90000E940610CF911F910F91FF90EF90DF901D
:105EA000CF90BF90AF909F908F90089560E070E08A
:105EB0008FE793E420912103309122034091230343
:105EC000509124030E94E550DC01CB018093B20580
:105ED0009093B305A093B405B093B5050895FC0164
:105EE000EA54FA4F808190E00895CF93DF93EC015C
:105EF000662351F1E1E1FEE007C09091C00095FFFB
:105F0000FCCF8093C600319684918823B1F78EEE42
:105F100095E070E04AE050E00E94D335E8E1FEE011
:105F200007C09091C00095FFFCCF8093C6003196CA
:105F300084918823B1F78091C00085FFFCCF8AE06F
:105F40008093C6000E94B119BE01882777FD809515
:105F5000982F0E9480512FE632E143E050E40E94E6
:105F6000B35320E030E040E851E40E94B3530E9474
:105F70004D51CB01DF91CF91089580E090E00895DD
:105F8000CF93DF93EC01662351F1E1E1FEE007C01E
:105F90009091C00095FFFCCF8093C600319684910C
:105FA0008823B1F78EEE95E070E04AE050E00E9461
:105FB000D335E4E3FEE007C09091C00095FFFCCF2D
:105FC0008093C600319684918823B1F78091C000F8
:105FD00085FFFCCF8AE08093C6000E94B119BE0104
:105FE000882777FD8095982F0E94805120E030E02F
:105FF0004AEF5EE30E94B35320E030E040E85DE307
:106000000E94B35320E030E040E050E00E94055091
:10601000462F572F682F792FCB01BA01DF91CF91EF
:1060200008952F923F924F925F926F927F928F923C
:106030009F92AF92BF92CF92DF92EF92FF920F9317
:106040001F93CF93DF9300D00F92CDB7DEB780912F
:10605000B705882309F4EDC18FB7F8941092B705FE
:106060008FBF8091AC059091AD0560E00E94C02F7C
:106070002B013C016091A6057091A7058091A805B0
:106080009091A905A30192010E940450C62EB72E3B
:10609000182F092F9801862F9B2DA32FB22F8093A5
:1060A000B8059093B905A093BA05B093BB05BC01A0
:1060B000CD0120E030E040E251E40E94E1521816A8
:1060C0000CF450C198018C2D9B2DA32FB22FBC0135
:1060D000CD0120E030E040E251EC0E94DE5087FD2F
:1060E0003DC18091BC05882309F029C198018C2D00
:1060F0009B2DA32FB02FBC01CD0120912503309102
:10610000260340912703509128030E94B3536983CB
:106110007A831C01472F862F942FA22DB32D8093B5
:10612000C1059093C205A093C305B093C40598011F
:106130008C2D9B2DA32FB02FBC01CD012091BD052F
:106140003091BE054091BF055091C0050E94055099
:10615000B62EA72E982E892E0091C5051091C60542
:106160002091C7052C838091C8058B83A5019401DC
:10617000852F942FA32FB22FBC01CD013C812B8101
:10618000C02ED12EE32EF22EA70196010E94DE50E2
:1061900087FFB3C03C812B81802F912FA32FB22F7B
:1061A0008093BD059093BE05A093BF05B093C00535
:1061B000BC01CD01209121033091220340912303A2
:1061C000509124030E94B3536B83872E182F092FFD
:1061D0009801862F982DA32FB22F8093C9059093F5
:1061E000CA05A093CB05B093CC05C301B2012091A1
:1061F000CD053091CE054091CF055091D0050E943C
:10620000045020911D0330911E0340911F035091B3
:1062100020030E94B35320ED3CEC4CE45DE30E946C
:10622000B3536B017C016091D1057091D2058091CF
:10623000D3059091D40523E333E343E75FE30E9462
:10624000B3539B01AC01C701B6010E940550B62EA5
:10625000C72EA82E992E862F9C2DAA2DB92D80935E
:10626000D1059093D205A093D305B093D405409265
:10627000CD055092CE056092CF057092D005598120
:106280004A81852F942FA22DB32DBC01CD01FB8116
:10629000A8010F2F182D252F342FA90198010E9436
:1062A00005500B2D1C2D2A2D392DA90198010E9476
:1062B0000450C62EB72E182F092F9801862F9B2D1C
:1062C000A32FB22FBC01CD0120E030E040E050E030
:1062D0000E94DE5087FD4EC098018C2D9B2DA32F70
:1062E000B22FBC01CD0120E030E04FE753E40E9423
:1062F000E15218160CF042C038C00091B20510915E
:10630000B305E091B405EC83F091B505FB83A501DD
:106310009401852F942FA32FB22FBC01CD01C02E45
:10632000D12EEE2EFF2EA70196010E94E1521816E3
:106330000CF430CF0B2D1A2D9C828B822BCF80E05A
:1063400090E0A0E0B0E08093BD059093BE05A093DF
:10635000BF05B093C0051092BC05C8CE81E0809304
:10636000BC0508C081E08093BC05CC24BB241FE79A
:1063700003E404C0CC24BB2410E000E08091AC0511
:106380009091AD052091D5053091D6052817390794
:106390001CF01092B60514C02091290330912A03F5
:1063A00082179307B4F798018C2D9B2DA32FB02F44
:1063B000BC01CD010E944D51759567956093B6055E
:1063C0000E94304FDC01CB014091D7055091D80598
:1063D0006091D9057091DA05841B950BA60BB70B5C
:1063E000883823E1920720E0A20720E0B20708F1F5
:1063F0000E94304FDC01CB018093D7059093D805E4
:10640000A093D905B093DA058091AA059091AB05C8
:10641000181619066CF4EFE38F3F9E074CF4209199
:10642000AE053091AF058217930714F4A59A01C009
:10643000A5980F900F900F900F90DF91CF911F9123
:106440000F91FF90EF90DF90CF90BF90AF909F9013
:106450008F907F906F905F904F903F902F90089516
:1064600060E070E080E090E0089580E090E0A0E0DF
:10647000B0E08093C5059093C605A093C705B0937F
:10648000C80560E070E08FE793E42091210330912C
:10649000220340912303509124030E94E550DC0124
:1064A000CB018093B2059093B305A093B405B0934C
:1064B000B5056C9A6D9A9D9AE1E0F1E0808180616A
:1064C000808387ED80937A0010927E00EDE7F0E004
:1064D000108280818160808380818260808380815E
:1064E0008460808380E888BDEEE6F0E0808184608F
:1064F00080836AEF70E080E090E00E946C4F85E05E
:1065000090E060E00E94752F9093D6058093D505AA
:1065100083E191E060E00E94752F90932A038093BD
:1065200029030895089580E090E060E00E94752FAF
:1065300080E090E0A0E0B0E08093A6059093A705EE
:10654000A093A805B093A9051092AF051092AE05CF
:106550001092B1051092B0051092B60582E060E08D
:106560000E94AF4E1092B3051092B2051092B7057B
:1065700083E060E00E94AF4E1092AF051092AE052E
:1065800084E060E00E94AF4E0895CF93C82F82E070
:1065900060E00E94AF4EE1E1FEE007C09091C000D4
:1065A00095FFFCCF8093C600319684918823B1F784
:1065B0008EEE95E06C2F40E050E00E949635809181
:1065C000C00085FFFCCF8AE08093C600E1E5FEE0D5
:1065D00007C09091C00095FFFCCF8093C600319614
:1065E00084918823B1F78091C00085FFFCCF8AE0B9
:1065F0008093C600CF910895CF93C82F82E060E0CA
:106600000E94AF4EE1E1FEE007C09091C00095FF0F
:10661000FCCF8093C600319684918823B1F78EEE2B
:1066200095E06C2F40E050E00E9496358091C000CC
:1066300085FFFCCF8AE08093C600EEE7FEE007C04E
:106640009091C00095FFFCCF8093C6003196849155
:106650008823B1F78091C00085FFFCCF8AE080934A
:10666000C600CF9108951F920F920FB60F920BB6EE
:106670000F9211242F933F934F935F936F937F93C8
:106680008F939F93AF93BF93EF93FF9380912B03CF
:10669000882331F48091B6058093DB058111749ACB
:1066A0009091DB0580912B03891708F074988F5F18
:1066B0008F7780932B038091DC05833009F44CC0E5
:1066C000843028F48130E9F08230C8F50DC085307F
:1066D00009F46BC0853008F45BC0863009F481C0D2
:1066E000873009F087C07FC088E080937B0080E41A
:1066F00080937C0080917A00806480937A0081E0AE
:106700001BC0409178005091790060E070E080916A
:10671000DD059091DE05A091DF05B091E005840FC5
:10672000951FA61FB71F8093DD059093DE05A093EC
:10673000DF05B093E00582E08093DC055BC088E074
:1067400080937B0082E480937C0080917A00806457
:1067500080937A0083E0F0CF4091780050917900E7
:1067600060E070E08091E1059091E205A091E30581
:10677000B091E405840F951FA61FB71F8093E10514
:106780009093E205A093E305B093E40584E0D4CFB1
:1067900088E080937B0081E480937C0080917A0084
:1067A000806480937A0085E0C7CF40917800509153
:1067B000790060E070E08091E5059091E605A09198
:1067C000E705B091E805840F951FA61FB71F8093BA
:1067D000E5059093E605A093E705B093E80586E00C
:1067E000ABCF87E0A9CF1092DC058091E9058F5FE0
:1067F0008093E9058091E905803108F45DC020911E
:10680000DD053091DE053093AD052093AC058FEFAB
:106810009FE34091E1055091E205841B950B909315
:10682000AB058093AA0581E08093B7051092E90536
:106830001092DD051092DE051092DF051092E00542
:106840001092E5051092E6051092E7051092E80512
:106850001092EA051092EB051092EC051092ED05EE
:106860001092E1051092E2051092E3051092E40502
:106870008091290390912A03281739074CF0109230
:10688000B1051092B00580E00E94C5320E94B11996
:106890002091AC053091AD058091D5059091D6053C
:1068A000821793074CF01092B1051092B00580E06A
:1068B0000E94FC320E94B119FF91EF91BF91AF91FC
:1068C0009F918F917F916F915F914F913F912F9108
:1068D0000F900BBE0F900FBE0F901F9018951F9238
:1068E0000F920FB60F920BB60F9211242F933F9376
:1068F0004F935F936F938F939F93EF93FF93609169
:10690000C60020916F0630917006C90101968F77FD
:10691000907040917106509172068417950741F06E
:1069200021513A4FF90160839093700680936F066E
:10693000FF91EF919F918F916F915F914F913F9157
:106940002F910F900BBE0F900FBE0F901F901895B8
:106950000F931F939A01AB01203081EE380780E03E
:10696000480780E0580769F182E08093C00060E04A
:1069700079E08DE390E00E94CD5489019A010150A5
:10698000104020403040C901B80122E030E040E032
:1069900050E00E94CD543093C5002093C4008091F4
:1069A000C10080618093C1008091C10088608093A4
:1069B000C1008091C10080688093C1001F910F9138
:1069C00008951092C00020E130E0E5CF20917106DB
:1069D0003091720680916F0690917006821793072E
:1069E00071F0F901E151FA4F80812F5F3F4F2F770E
:1069F0003070309372062093710690E008958FEF07
:106A00009FEF0895809171069091720690937006A1
:106A100080936F0608956F927F928F929F92AF92AC
:106A2000BF92CF92DF92EF92FF920F931F93CF937B
:106A3000DF93CDB7DEB7A0970FB6F894DEBF0FBED9
:106A4000CDBF3C01DB01CA0141155105610571054E
:106A500051F4C30140E350E060E070E020E030E03A
:106A60000E949E3541C08E010F5F1F4FCC24DD2454
:106A70007601822E9924AA24BB24BC01CD01A50154
:106A800094010E94AB54F80161938F010894C11CDA
:106A9000D11CE11CF11CC901DA010097A105B10567
:106AA00061F714C0E1E0F0E0EC0FFD1FEC0DFD1DFF
:106AB00040814A3010F4405D01C0495C50E060E024
:106AC00070E0C30120E030E00E949E350894C108C8
:106AD000D108E108F108FFEFCF16FFEFDF06FFEF67
:106AE000EF06FFEFFF06F1F6A0960FB6F894DEBFB3
:106AF0000FBECDBFDF91CF911F910F91FF90EF900F
:106B0000DF90CF90BF90AF909F908F907F906F90CD
:106B100008952115310539F48091C00085FFFCCF1F
:106B20004093C60008950E940B3508959A01462FA0
:106B300050E060E070E00E9489350895CF92DF92C6
:106B4000EF92FF92CF93DF93EC016A017B01211555
:106B5000310539F48091C00085FFFCCFC092C6009A
:106B60001BC02A303105B1F477FF10C04DE250E070
:106B700060E070E020E030E00E949E35F094E09408
:106B8000D094C094C11CD11CE11CF11CCE01B701F2
:106B9000A6012AE00E940B35DF91CF91FF90EF9084
:106BA000DF90CF9008959A01FB01AF01662757FD52
:106BB0006095762F0E949E350895CF93DF93EC0168
:106BC0004DE050E060E070E020E030E00E949E3553
:106BD000CE014AE050E060E070E020E030E00E944A
:106BE0009E35DF91CF910895CF93DF93EC019A0109
:106BF000AB0160E070E00E948935CE010E94DD3576
:106C0000DF91CF9108958F929F92BF92CF92DF92A2
:106C1000EF92FF920F931F93CF93DF934C016A0182
:106C20007B01B22ECB01BA0120E030E040E050E021
:106C30000E94DE5087FF0DC0C4014DE250E060E0CD
:106C400070E020E030E00E949E35F7FAF094F7F80B
:106C5000F094C0E050E040E030E02FE313C0FA01D0
:106C6000B9018F2F942FA72FB22FBC01CD0120E0A7
:106C700030E040E251E40E94E550562F472F382F74
:106C8000292FCF5FCB1559F7C701B601DA01F901FA
:106C90000B2F142F2F2F3E2FA90198010E94055072
:106CA0006B01E82EC92F862F9D2DAE2DBC2FBC0168
:106CB000CD010E945251D62F172F082FF92E0E9476
:106CC0007E519B01AC018C2D9D2DAE2DBC2FBC01A6
:106CD000CD010E940450D62EE72EC82FC92EC40124
:106CE0004D2F512F602F7F2D2AE030E00E948935F3
:106CF000BB2009F446C0E5EFF2E006C09091C00069
:106D000095FFFCCF8093C60081918823B9F739C0E5
:106D10008D2D9E2DAC2FBC2DBC01CD0120E030E08F
:106D200040E251E40E94B353EB01182F092F980160
:106D3000862F9D2FA32FB22FBC01CD010E944D5154
:106D40006B017C01EE24D7FCE094FE2CC401B7015A
:106D5000A6012AE030E00E949E35C701B6010E94DC
:106D600080519B01AC01B8018C2F9D2FA72FB62F0E
:106D7000BC01CD010E940450D62EE72EC82FC92E8B
:106D8000BA94BB2029F6DF91CF911F910F91FF900C
:106D9000EF90DF90CF90BF909F908F9008950E94CA
:106DA000033608952F923F924F925F926F927F9297
:106DB0008F929F92AF92BF92CF92DF92EF92FF920B
:106DC0000F931F93CF93DF93CDB7DEB7C055D0405D
:106DD0000FB6F894DEBF0FBECDBF2C017A8F698F3E
:106DE0004A012CA708AFE9AEAAAEBBAECCAEDDAE71
:106DF000022F10E0000F111F000F111F9A01200F2A
:106E0000311F3BAB2AABD9018D919D910D90BC9167
:106E1000A02D898B9A8BAB8BBC8BF201E00FF11FFD
:106E2000BC01CD0120813181428153810E940550F6
:106E30006EAF7FAF21968FAF219722969FAF22979B
:106E4000B8ADEB2EFF24EE0CFF1CEE0CFF1CF40182
:106E5000EE0DFF1DFDABECAB80809180A280B38076
:106E6000F201EE0DFF1DC501B40120813181428187
:106E700053810E94055023966FAF239724967FAFCE
:106E8000249725968FAF259726969FAF2697F9AD25
:106E90008F2F90E0880F991F880F991FF201E80F3C
:106EA000F91F20813181428153812B8F3C8F4D8F7F
:106EB0005E8FE98DFA8DE80FF91F60817181828103
:106EC00093810E940450462F572F682F792F4F8FA0
:106ED00058A369A37AA3A98DBA8D1C968D919D9113
:106EE0000D90BC91A02D8EA79FA7A8ABB9ABD201E6
:106EF0001C962D913D914D915C911F972FA338A722
:106F000049A75AA729893A894B895C895058298B06
:106F10003A8B4B8B5C8BD501C401B0588D8B9E8B0B
:106F2000AF8BB88FE98DFA8DE00FF11F6081718111
:106F300082819381FEADEFAD21965FAD21972296C0
:106F40004FAD22970F2F1E2F252F342FA901980107
:106F50000E9404506B01482E792EE98DFA8DEE0DBA
:106F6000FF1D60817181828193812396FFAD2397FC
:106F70002496EFAD249725965FAD259726964FADC5
:106F800026970F2F1E2F252F342FA90198010E941D
:106F90000450F62EE72E682E592E69897A898B893E
:106FA0009C89F7010F2F1E2F262D352DA901980141
:106FB0000E94B3534B015C016D897E898F89988D46
:106FC0000C2D1D2D242D372DA90198010E94B3539E
:106FD0009B01AC01C501B4010E9404506BA37CA3CA
:106FE0008DA39EA369897A898B899C89242D372D4D
:106FF000A90198010E94B3534B015C016D897E8900
:107000008F89988DF7010F2F1E2F262D352DA90161
:1070100098010E94B3539B01AC01C501B4010E94C9
:1070200005509B01AC016BA17CA18DA19EA10E948A
:107030007850162F072FF82EE92EA8019701852FDB
:10704000942FA32FB22FBC01CD0120E030E040E00F
:1070500050E00E94DE5087FF12C0A8019701852FE3
:10706000942FA32FB22FBC01CD012BED3FE049ECB3
:1070700050E40E940550162F072FF82EE92EAB96EC
:107080008FADAB97882391F0A8019701852F902FA2
:10709000A32FBE2DBC01CD012BED3FE049EC50E408
:1070A0000E940450162F072FF82EE92EA8019701F1
:1070B000852F902FA32FBE2DBC01CD01AA962CADFC
:1070C0003DAD4EAD5FADAA970E94B3532F8D38A151
:1070D00049A15AA15F770E94EE524B015C012FE655
:1070E00032E143E85AE30E94DE5087FD62C2C501E7
:1070F000B4010E94BB510E945251DC01CB019FABF5
:107100008EABBC0180E090E00E947E514B015C019F
:10711000A8019701852F902FA32FBE2DBC01CD0173
:10712000A50194010E94E550362E272E8BA39BA724
:107130006F8D78A189A19AA1A50194010E94E550C3
:107140002A966FAF2A972B967FAF2B972C968FAFEF
:107150002C972D969FAF2D976EA57FA588A999A9ED
:107160002FA138A549A55AA50E940450A501940154
:107170000E94E5502E966FAF2E972F967FAF2F97D8
:1071800060968FAF609761969FAF6197A1013BA119
:107190002BA5852F942FA32FB22FBC01CD0120E06A
:1071A00030E040E05FE30E94B353F1015BA14BA5E7
:1071B0000F2F1E2F252F342FA90198010E94B353A2
:1071C0009B01AC0160E070E080E89FE30E94045006
:1071D0006EA727967FAF279728968FAF2897299677
:1071E0009FAF2997B9ADEB2FF0E0EE0FFF1FEE0F29
:1071F000FF1FCE010196E80FF91F2B8D3C8D4D8DA1
:107200005E8D20833183428353832FA138A549A506
:107210005AA52D873E874F87588B882441E050E040
:1072200058A74FA3BCA5AB2FB0E0AA0FBB1FAA0F56
:10723000BB1F9C012A0F3B1F3C8F2B8F58AD452F46
:1072400050E0440F551F440F551F81E090E08C0F14
:107250009D1F840F951F98A38F8FFDA7ECA788C152
:1072600098E198150CF46FC069897A898B899C899B
:10727000432D522DEBA1FBA58A019F01A901980185
:107280000E94B3536B017C016D897E898F89988D33
:107290004EA527965FAD27972896EFAD289729969C
:1072A000FFAD29978A019F01A90198010E94B3535C
:1072B0009B01AC01C701B6010E940550762E672ED6
:1072C000582E492E69897A898B899C892896EFAD39
:1072D00028972996FFAD29979F01A90198010E943F
:1072E000B353F62EE72ED82EC92E6D897E898F894D
:1072F000988D432D522DEBA1FBA58A019F01A90179
:1073000098010E94B3539B01AC01F701B6018F2F86
:107310009E2FA72FB62FBC01CD010E940450462FEF
:10732000572F682F792F498B5A8B6B8B7C8B8394CB
:10733000A3019201852F942FA32FB22F8D8B9E8BAB
:10734000AF8BB88F81C0AFA1B8A5BD0180E090E040
:107350000E947E51432D522DEBA1FBA58A019F0176
:10736000A90198010E94B353162F072FF82EE92E7A
:10737000A8019701852F942FA32FB22FBC01CD0117
:107380000E94E2506D8B7E8B8F8B988FA8019701A6
:10739000852F942FA32FB22FBC01CD010E9416542C
:1073A0002B013C01EAA9FBA980819181A281B381D3
:1073B0006C017D01F7FAF094F7F8F094ACA9BDA93F
:1073C0008D909D90AD90BC90C701B6012D893E89EE
:1073D0004F89588D0E94B353698B7A8B8B8B9C8B12
:1073E000C501B401A30192010E94B3539B01AC01FA
:1073F00069897A898B899C890E940550AB01682F25
:10740000792F498B5A8B6B8B7C8BC701B601A301FB
:1074100092010E94B3536B017C01C501B4012D8917
:107420003E894F89588D0E94B3539B01AC01C7011F
:10743000B6010E940450462F572F682F792F4D8B8D
:107440005E8B6F8B788F88245EAD4FAD21963FADFC
:10745000219722962FAD2297852F942FA32FB22FFD
:10746000BC01CD0129893A894B895C890E9405506C
:10747000DC01CB01EB8DFC8D80839183A283B383F0
:1074800023965FAD239724964FAD249725963FAD65
:10749000259726962FAD2697852F942FA32FB22FB1
:1074A000BC01CD012D893E894F89588D0E94055020
:1074B000DC01CB01EF8DF8A180839183A283B3839C
:1074C000ACA5BDA56D917D918D919C912A964FADF6
:1074D0002A972B965FAD2B972C96EFAD2C972D9678
:1074E000FFAD2D978A019F01A90198010E940550C7
:1074F000DC01CB01ECA5FDA580839183A283B3833E
:107500006D857E858F8598892E964FAD2E972F9607
:107510005FAD2F976096EFAD60976196FFAD619775
:107520008A019F01A90198010E940550DC01CB014D
:107530008D879E87AF87B88BCE010196BE016B5FAA
:107540007F4FAE01475F5F4F9E01235F3F4FEAAC25
:10755000FBAC0CAD1DADFBE6CF2ED12CCC0EDD1E51
:107560000E94B93F2FA138A52F5F3F4F38A72FA307
:107570004FA158A58EA99FA94817590708F470CEA6
:10758000698D7A8D6C5F7F4F498D5A8D485F5F4F53
:10759000298D3A8D245F3F4F898D9A8DEAACFBACE3
:1075A0000CAD1DADEBE6CE2ED12CCC0EDD1E0E9417
:1075B000B93FC05BDF4F0FB6F894DEBF0FBECDBF43
:1075C000DF91CF911F910F91FF90EF90DF90CF90BF
:1075D000BF90AF909F908F907F906F905F904F90F3
:1075E0003F902F9008952F923F924F925F926F920B
:1075F0007F928F929F92AF92BF92CF92DF92EF9243
:10760000FF920F931F93CF93DF93CDB7DEB76897A9
:107610000FB6F894DEBF0FBECDBF1C016A017B011F
:1076200028013901DC01D8966D917D918D919C9155
:10763000DB970E947E514B015C01A70196010E94DD
:10764000B3530E94CB500E94525169837A838B833B
:107650009C83C501B401A30192010E94B3530E940F
:10766000CB500E9452516D837E838F8398872981EE
:107670003A814B815C81283731054105510540F441
:1076800088E790E0A0E0B0E089839A83AB83BC8375
:107690002D813E814F81588528373105410551059F
:1076A00040F488E790E0A0E0B0E08D839E83AF8354
:1076B000B887F101EC5BFF4F40805180628073809E
:1076C000D101DC966D917D918D919C91DF970E9407
:1076D0007E516D877E878F87988BC301B2010E9490
:1076E000805169877A878B879C8720E030E040E073
:1076F00050E00E94DE50882339F1C501B401A50194
:1077000094010E94B3536B017C016D857E858F854A
:1077100098899B01AC010E94B3539B01AC01C70146
:10772000B6010E9404506B017C0169857A858B85C6
:107730009C859B01AC010E9405509B01AC01C701D7
:10774000B6010E94E55004C060E070E080E090E087
:10775000382F292F862F972FA32FB22FBC01CD01B1
:107760000E94CB500E944D516B017C01F101E05C05
:10777000FF4F60817181828193810E947E51698B6C
:107780007A8B8B8B9C8B66277727CB0164197509C5
:10779000860997090E9480512B013C0120E030E0CE
:1077A00040E050E00E94DE50882349F169897A89DF
:1077B0008B899C899B01AC010E94B3536D8B7E8B9E
:1077C0008F8B988FC501B401A50194010E94B3531A
:1077D0009B01AC016D897E898F89988D0E94045030
:1077E0004B015C01C301B201A30192010E9405504B
:1077F0009B01AC01C501B4010E94E55004C060E0EA
:1078000070E080E090E0382F292F862F972FA32F4C
:10781000B22FBC01CD010E94BB51F10140885188BB
:1078200062887388530142018C189D08AE08BF0816
:107830000E944D51DC01CB01A5019401281B390B9D
:107840004A0B5B0BDA01C90157FF76C069857A855F
:107850008B859C8520E030E040E050E00E94DE50C7
:10786000882309F447C069857A858B859C859B01AF
:10787000AC010E9405506B017C01C301B2010E9462
:107880007E519B01AC01C701B6010E94B3536B014D
:107890007C016D857E858F8598899B01AC010E9456
:1078A000B3539B01AC01C701B6010E9404506B01A8
:1078B0007C0169897A898B899C899B01AC010E9432
:1078C000B3539B01AC01C701B6010E9405506B0187
:1078D0007C0169857A858B859C8520E030E040E8D5
:1078E00050E40E94B3539B01AC01C701B6010E9452
:1078F000E55004C060E070E080E090E0382F292F70
:10790000862F972FA32FB22FBC01CD010E94CB5001
:107910000E944D516B017C01F7FE03C0CC24DD2495
:107920007601C414D504E604F70410F07301620173
:1079300080E090E0A0E0B0E02FB7F894F101E45BC4
:10794000FF4F3081332309F5F101C48AD58AE68AD5
:10795000F78A8C0D9D1DAE1DBF1D808F918FA28F4C
:10796000B38F89819A81AB81BC8184AF95AFA6AF7B
:10797000B7AFA101405C5F4F8D819E81AF81B8851B
:10798000FA0180839183A283B3832FBF68960FB6D9
:10799000F894DEBF0FBECDBFDF91CF911F910F9145
:1079A000FF90EF90DF90CF90BF90AF909F908F901F
:1079B0007F906F905F904F903F902F9008954F92DF
:1079C0005F926F927F928F929F92AF92BF92CF926F
:1079D000DF92EF92FF920F931F93CF93DF93EB0110
:1079E0006A01209709F47DC04115510509F479C059
:1079F0007AA46BA45CA44DA46EA17FA188A599A5CF
:107A0000F301A2010F2F1E2F252F342FA90198015A
:107A10000E94DE50882309F464C08FA9882309F0EE
:107A200054C0F601C6A0D7A0E0A4F1A4A30192011E
:107A3000852F942FA32FB22FBC01CD01A701960152
:107A40000E94E15218160CF040C0C701B601A70110
:107A500096010E94B3536B017C018AA99BA9ACA932
:107A6000BDA99C01AD015058CA01B9010E94055041
:107A70002EA53FA548A959A90E94B3539B01AC016B
:107A8000C701B6010E9404500E942054162FC72E31
:107A9000082FF92EA3019201852F942FA32FB22F27
:107AA000BC01CD01812E9C2CA02EBF2CA5019401E0
:107AB0000E94DE5087FF04C0172DC62C052DF42C24
:107AC000512F4C2D302F2F2D02C0A3019201852F55
:107AD000942FA32FB22F8EA39FA3A8A7B9A781E0AD
:107AE0008EABDF91CF911F910F91FF90EF90DF90C0
:107AF000CF90BF90AF909F908F907F906F905F904E
:107B00004F900895CF92DF92EF92FF920F931F93C1
:107B1000CF9380917506809175062091740690E050
:107B2000821B91098F709070843091052CF1C09167
:107B30007506C350CF7040E050E0EE24FF248DE482
:107B4000C82ED12C15C0CC2309F4C0E1C1508C2F14
:107B500090E08C9D80018D9D100D9C9D100D112439
:107B60000A58194FC801B7010E94DF3CA7017801EC
:107B700080917406C81739F7CF911F910F91FF902C
:107B8000EF90DF90CF9008956F927F928F929F92A7
:107B9000AF92BF92CF92DF92EF92FF920F931F931B
:107BA000CF93DF93EC013B01009709F473C08FA9D9
:107BB000882309F06FC0CEA0DFA0E8A4F9A4FB01E0
:107BC000B6A0A7A090A481A4C701B601F501A401A5
:107BD0000F2F1E2F252F342FA90198010E94DE5050
:107BE00087FF58C0C701B601A70196010E94B35391
:107BF0006B017C018AA99BA9ACA9BDA99C01AD011F
:107C00005058CA01B9010E9405502EA53FA548A9A8
:107C100059A90E94B3539B01AC01C701B6010E9450
:107C200004500E942054C62EC72FD82FF92EA5012C
:107C30009401852F942FA32FB22FBC01CD010C2DC1
:107C40001C2F2D2F3F2DA90198010E94DE5087FF88
:107C500004C0CB2CCA2DD92DF82CA5019401852F59
:107C60009A2DA32FB82DBC01CD010C2D1C2F2D2F2B
:107C70003F2DA90198010E94DE50882359F0802FE2
:107C80009C2FAD2FBF2DF30186A397A3A0A7B1A76B
:107C900081E086ABDF91CF911F910F91FF90EF9024
:107CA000DF90CF90BF90AF909F908F907F906F901C
:107CB0000895CF92DF92EF92FF920F931F93CF938D
:107CC000C0917406EE24FF2420E030E09DE4C92E2C
:107CD000D12C16C08C2F90E08C9D80018D9D100DB5
:107CE0009C9D100D11240A58194FC901B701A80114
:107CF0000E94C43DCF5FC03109F4C0E09701780114
:107D000080917506C81731F7C901B70140E050E00E
:107D10000E94C43DCF911F910F91FF90EF90DF9093
:107D2000CF9008952F923F924F925F926F927F92E1
:107D30008F929F92AF92BF92CF92DF92EF92FF927B
:107D40000F931F93CF93DF93F0907406C0E0D0E0C1
:107D50002DE4222E312C39C0229D6001239DD00CB0
:107D6000329DD00C112486E796E0C80ED91E2097CC
:107D700031F18EA9882321F4F60186A98823F9F030
:107D80008AA09BA0ACA0BDA06EA17FA188A599A54B
:107D9000A50194010E94E5502B013C01F60166A16A
:107DA00077A180A591A5A50194010E94E5508B01C2
:107DB0009C01CE01B301A2010E94F33A1EAAF394E2
:107DC000F0E1FF1609F4FF24E6012F2D332727FDEC
:107DD00030958091750690E02817390709F0BCCFDF
:107DE0002097F1F0CAA0DBA0ECA0FDA06EA17FA1BE
:107DF00088A599A5A70196010E94E5504B015C0159
:107E000060E070E080E090E4A70196010E94E550F8
:107E10008B019C01CE01B501A4010E94F33A1EAA78
:107E2000DF91CF911F910F91FF90EF90DF90CF9056
:107E3000BF90AF909F908F907F906F905F904F908A
:107E40003F902F9008950E94823D0E94593E0E94CB
:107E5000923E0895109275061092740680E1E6E451
:107E6000FBE0DF011D928A95E9F780E090E0A0E059
:107E7000B0E08093B60B9093B70BA093B80BB09380
:107E8000B90B8093BA0B9093BB0BA093BC0BB09330
:107E9000BD0B8093BE0B9093BF0BA093C00BB09310
:107EA000C10B8093C20B9093C30BA093C40BB093F0
:107EB000C50B8093C60B9093C70BA093C80BB093D0
:107EC000C90B0895CF939091740680917506981709
:107ED00071F1A09174062A2F30E08DE490E0289F84
:107EE000F001299FF00D389FF00D1124E254F94F55
:107EF000C081B0E017C02A2F30E0289FF001299FF1
:107F0000F00D389FF00D1124E254F94F408151815A
:107F100062817381411551056105710509F0BF5FEB
:107F2000AF5FAF7020917506A21729F70AC0609164
:107F3000B303662321F087E070E00E943E4DC0E06D
:107F4000B0E08091B303882339F4BB2329F487E0A0
:107F500060E070E00E943E4D8091B303882339F0C9
:107F6000CC2329F087E06C2F70E00E943E4DCF912A
:107F700008952F923F924F925F926F927F928F92CD
:107F80009F92AF92BF92CF92DF92EF92FF920F93A8
:107F90001F93CF93DF93CDB7DEB7C156D0400FB656
:107FA000F894DEBF0FBECDBF5C014B015CA34BA3B9
:107FB0003EA72DA73E2C5F2C602E412EDEAACDAA17
:107FC000809175068F5F803109F480E0282F332778
:107FD00027FD30956F963FAF2EAF6F9705C00E947B
:107FE000113081E00E94E0198091740690E06F9654
:107FF0004EAD5FAD6F978417950789F3D5016D91ED
:108000007D918D919C912091920B3091930B409199
:10801000940B5091950B0E94B3530E9483532A9660
:108020006FAF2A972B967FAF2B972C968FAF2C97FD
:108030002D969FAF2D97F40160817181828193818C
:108040002091960B3091970B4091980B5091990B82
:108050000E94B3530E9483532E966FAF2E972F9694
:108060007FAF2F9760968FAF609761969FAF6197B4
:10807000ABA1BCA16D917D918D919C9120919A0BAA
:1080800030919B0B40919C0B50919D0B0E94B353E0
:108090000E94835362966FAF629763967FAF639738
:1080A00064968FAF649765969FAF6597EDA5FEA523
:1080B000608171818281938120919E0B30919F0B11
:1080C0004091A00B5091A10B0E94B3530E94835387
:1080D0006DA77EA78FA798AB8091520B9091530B01
:1080E000A091540BB091550B2DA53EA54FA558A9B5
:1080F000281739074A075B0709F445C06091B403A4
:10810000E62FF0E0EE0FFF1FE455FA4F80819181DA
:108110000E94C02F20E030E04AE253E40E94DE508B
:1081200087FF31C080917306882369F54DA55EA550
:108130006FA578A94093520B5093530B6093540B47
:108140007093550BE5EEFEE007C09091C00095FFDF
:10815000FCCF8093C600319684918823B1F7EBEE73
:10816000FEE007C09091C00095FFFCCF8093C60051
:10817000319684918823B1F78091C00085FFFCCFB0
:108180008AE08093C6008091520B9091530BA0918E
:10819000540BB091550B2DA53EA54FA558A9281BF2
:1081A000390B4A0B5B0BDA01C90157FF07C0B095C9
:1081B000A095909581959F4FAF4FBF4FBC01CD01CA
:1081C0000E9480516B017C0160919E0B70919F0B0E
:1081D0008091A00B9091A10B20E030E04DEC53E496
:1081E0000E94B3539B01AC01C701B6010E94E1524A
:1081F00018166CF54DA55EA56FA578A94093520B96
:108200005093530B6093540B7093550BE5EEFEE0C7
:1082100007C09091C00095FFFCCF8093C6003196B7
:1082200084918823B1F7E5E0FFE007C09091C0009A
:1082300095FFFCCF8093C600319684918823B1F7D7
:108240008091C00085FFFCCF8AE08093C6008091BA
:10825000750690E02DE430E0829FB001839F700DA1
:10826000929F700D11246A58794F7CA36BA3FB0178
:10827000E45BFF4F10828091460B9091470BA091D9
:10828000480BB091490B8DA39EA3AFA3B8A72D9621
:108290008CAC9DACAEACBFAC2D97881A990AAA0ADB
:1082A000BB0AB7FE08C0B094A09490948094811C3F
:1082B000911CA11CB11CABA1BCA18D929D92AD9251
:1082C000BC92139720914A0B30914B0B40914C0B71
:1082D00050914D0B29A73AA74BA75CA76196CCAC50
:1082E000DDACEEACFFAC6197C21AD30AE40AF50A22
:1082F000F7FE08C0F094E094D094C094C11CD11C47
:10830000E11CF11CABA1BCA11496CD92DD92ED92C3
:10831000FC92179720914E0B30914F0B4091500BD0
:108320005091510B21962CAF3DAF4EAF5FAF2197CF
:1083300065968CAD9DADAEADBFAD6597821B930BC1
:10834000A40BB50BB7FF07C0B095A095909581958C
:108350009F4FAF4FBF4F782E292EA9AB6696BFAF68
:108360006697EBA1FCA180879187A287B3872091B4
:10837000520B3091530B4091540B5091550B29AF38
:108380003AAF4BAF5CAF2091FC023091FD028DA55E
:108390009EA5AFA5B8A949AD5AAD6BAD7CAD841B08
:1083A000950BA60BB70BB7FF07C0B095A09590959E
:1083B00081959F4FAF4FBF4F442737FD4095542FB6
:1083C000BC01CD010E94795424E630E040E050E049
:1083D0000E94CD5489019A01ABA1BCA11C960D93BA
:1083E0001D932D933C931F97872D922DA9A96696D7
:1083F000BFAD66978C159D05AE05BF0514F4D7017A
:10840000C60180179107A207B30714F4D901C80168
:10841000B501A40188169906AA06BB0614F4AC019E
:10842000BD01EBA1FCA1408B518B628B738B46305D
:1084300051056105710510F40C94CB4AE85BFF4FC0
:108440008091B30390E0A0E0B0E080839183A283A9
:10845000B383ABA1BCA190961C9290972D962CADA6
:108460003DAD4EAD5FAD2D976DA17EA18FA198A5BD
:1084700026173707480759071CF481E090968C931C
:1084800061968CAD9DADAEADBFAD619729A53AA506
:108490004BA55CA582179307A407B5074CF4ABA1C5
:1084A000BCA190968C919097826090968C939097B7
:1084B00065962CAD3DAD4EAD5FAD659721966CAD2B
:1084C0007DAD8EAD9FAD2197261737074807590719
:1084D0004CF4ABA1BCA190968C919097846090963F
:1084E0008C9390972DA53EA54FA558A969AD7AAD5F
:1084F0008BAD9CAD261737074807590744F4ABA14D
:10850000BCA190968C919097886090968C93EDA9E1
:10851000FEA98081ABA1BCA191968C939197811407
:108520009104A104B10409F01598EBA1FCA1848188
:108530009581A681B7810097A105B10509F017982B
:10854000EBA1FCA180859185A285B3850097A1054B
:10855000B10509F04298EBA1FCA184859585A6851B
:10856000B7850097A105B10509F0A098ABA1BCA102
:108570001C962D913D914D915C911F9769962CAF62
:108580003DAF4EAF5FAF69972115310541055105EC
:1085900049F4B090660BA090670B8090680B7090C8
:1085A000690B08C0B0907E0BA0907F0B8090800B71
:1085B0007090810B832D952DA62DB42DBC01CD017E
:1085C000F5010F2F1A2D282D372DA90198010E9492
:1085D000DE5087FD04C0B32CA52C862C742C909102
:1085E000750680917406E92FF0E0E81BF109EF7041
:1085F000F070FEABEDABBF01882777FD8095982F1B
:108600000E9480516B017C0120E030E040E051E4A9
:108610000E94DE5087FF20C02DA93EA922303105DF
:10862000DCF0A501852F9A2DA82DB72DBC01CD0119
:10863000A70196010E94B353462F572F682F792F19
:10864000CB01BA0120E030E040E05EE30E94B3538A
:10865000B62EA72E882E792E2D966CAD7DAD8EADC3
:108660009FAD2D972DA13EA14FA158A5621B730B65
:10867000840B950B0E9480512091920B3091930BAB
:108680004091940B5091950B0E94E550362E272E69
:108690008DA399ABA101382F292F852F942FA32FBC
:1086A000B22F898B9A8BAB8BBC8B61966CAD7DADF9
:1086B0008EAD9FAD619729A53AA54BA55CA5621B20
:1086C000730B840B950B0E9480512091960B309177
:1086D000970B4091980B5091990B0E94E550962E64
:1086E000672E582E492E9201862F962DA32FB22F3A
:1086F0008D8B9E8BAF8BB88F65966CAD7DAD8EAD3F
:108700009FAD659721962CAD3DAD4EAD5FAD2197E8
:10871000621B730B840B950B0E94805120919A0B66
:1087200030919B0B40919C0B50919D0B0E94E5500A
:1087300069A77DAF22968FAF229726969FAF269787
:10874000472F382F292F862F942FA32FB22F898FB1
:108750009A8FAB8FBC8F0091FC021091FD026DA52A
:108760007EA58FA598A929AD3AAD4BAD5CAD621B36
:10877000730B840B950B0E94805120919E0B3091BE
:108780009F0B4091A00B5091A10B0E94E5506B01F3
:108790007C01B801882777FD8095982F0E94805131
:1087A0009B01AC01C701B6010E94B35320E030E049
:1087B00048EC52E40E94E550162F072F382F292F3E
:1087C000462F572F682F792F6A017B014D8F5E8FBF
:1087D0006F8F78A3ABA1BCA14D915D916D917C9100
:1087E000139749AF5AAF6BAF7CAF41155105610587
:1087F000710581F514968D919D910D90BC91A02DE0
:108800000097A105B10531F5EBA1FCA1408551858B
:10881000628573854115510561057105D9F4412FB4
:10882000502F632F722FCB01BA0120E030E040E0DF
:1088300050E00E94E152181624F0F7FAF094F7F88D
:10884000F094ABA1BCA19E96CD92DD92ED92FC92EC
:10885000D19745C0A1013DA129A9852F922DA32F14
:10886000B22FBC01CD010E945E546B017C019201CC
:10887000892D962DA32FB42DBC01CD010E945E54ED
:108880009B01AC01C701B6010E940550162F072FAE
:10889000C82E992E59A54DAD22963FAD229726960A
:1088A0002FAD2697852F942FA32FB22FBC01CD017A
:1088B0000E945E549B01AC01F8018F2F9E2FAC2DBE
:1088C000B92DBC01CD010E9405500E942054DC014D
:1088D000CB01EBA1FCA186A797A7A0ABB1ABABA145
:1088E000BCA19E962D913D914D915C91D197219681
:1088F0002CAF3DAF4EAF5FAF219760E070E080E8F6
:108900009FE30E94E5509B01AC01F5018F2F9A2D4A
:10891000A82DB72DBC01CD010E94B353C62EB72E92
:10892000A82E992E21966CAD7DAD8EAD9FAD219771
:108930000C2D1B2D2A2D392DA90198010E94B3530E
:108940006A966FAF6A97A0967FAFA097A1968FAFF8
:10895000A197A2969FAFA297472F382F292F862F36
:10896000942FA32FB22FEBA1FCA182A393A3A4A3C6
:10897000B5A360897189828993890E947E516DA314
:108980007EA38FA398A72A2D392DA90198010E94B3
:10899000B3530E94CB500E94525125966CAF7DAFCD
:1089A0008EAF9FAF2597ABA1BCA1D8966D937D9359
:1089B0008D939C93DB970F2EF1E16F2E7724F02D92
:1089C0006C0E7D1EFE013196FAA7E9A70F2EF1E28B
:1089D0002F2E3324F02D2C0E3D1E2F01D3016D912F
:1089E0007D918D919D913D014C2D5B2DEA2DF92DB1
:1089F0008A019F01A90198010E94B353DC01CB01B8
:108A0000F20181939193A193B1932F0162147304A6
:108A100029F722EA3BE03AAB29ABAE014F5E5F4F4C
:108A20005AA349A327963FAF2EAF279729A43AA46C
:108A3000BB24AA2460E8962E7FE3872ED101CD9037
:108A4000DD90ED90FD901D0111E0C701B60120E021
:108A500030E040E050E00E94E15218162CF010E0A7
:108A6000C701B601905802C0C701B6012796EEAD06
:108A7000FFAD279741905190619071902796FFAF7D
:108A8000EEAF2797A30192010E94E15218163CF520
:108A9000A7019601112309F45058C301B2010E94A5
:108AA000E5509B01AC016B2D7A2DE92DF82DCB0102
:108AB000DF01BC01CD010E94DE5087FD10C01123F3
:108AC00021F4F7FAF094F7F8F094C301B201A7018A
:108AD00096010E94E550B62EA72E982E892E29A128
:108AE0003AA12216330609F0A9CFA5019401852FDA
:108AF0009A2DA32FB82DBC01CD0120E030E040E835
:108B00005FE30E94DE5087FFABC029A43AA4D101E5
:108B1000CD90DD90ED90FD901D0111E0C701B601F3
:108B200020E030E040E050E00E94E15218162CF0C6
:108B300010E0C701B601905802C0C701B601E9A90B
:108B4000FAA94190519061907190FAABE9ABA30101
:108B500092010E94E15218163CF5A70196011123DB
:108B600009F45058C301B2010E94E5509B01AC01C9
:108B70006B2D7A2DE92DF82DCB01DF01BC01CD0144
:108B80000E94DE5087FD10C0112321F4F7FAF09403
:108B9000F7F8F094C301B201A70196010E94E550D5
:108BA000B62EA72E982E892E29A13AA12216330679
:108BB00009F0ADCF34E0C32EA9A5BAA56D917D9182
:108BC0008D919C910B2D1A2D292D382DA9019801DD
:108BD0000E94B353DC01CB01E9A5FAA581939193DF
:108BE000A193B193FAA7E9A7CA9431F76A965FAD4A
:108BF0006A97A0964FADA097A1963FADA197A29678
:108C00002FADA297852F942FA32FB22FBC01CD019A
:108C1000A401252F342FA90198010E94B353DC0130
:108C2000CB01EBA1FCA182A393A3A4A3B5A325969A
:108C30006CAD7DAD8EAD9FAD25970E947E51A40198
:108C4000252F342FA90198010E94B3530E9452513D
:108C5000DC01CB01EBA1FCA180AF91AFA2AFB3AF20
:108C60006DA17EA18FA198A521962CAD3DAD4EADF5
:108C70005FAD21970E94E550762E672E582E492E23
:108C800029AD3AAD4BAD5CAD21153105410551051E
:108C9000A1F5EBA1FCA184819581A681B781009704
:108CA000A105B10551F580859185A285B385009711
:108CB000A105B10511F5A3019201852F942FA32FD2
:108CC000B22FBC01CD012091760B3091770B4091F2
:108CD000780B5091790B0E94B3530E94CB500BA19B
:108CE0001CA10C5B1F4F0E945251DC01CB01F8010B
:108CF00080839183A283B38301C1A3019201852F55
:108D0000962DA32FB42DBC01CD0120917A0B30916B
:108D10007B0B40917C0B50917D0B0E94B3530E94C2
:108D2000CB500E9452510BA11CA10C5B1F4FD801CC
:108D30006D937D938D939C9313978090560B909099
:108D4000570BA090580BB090590B0E947E516B01AD
:108D50007C0169AD7AAD8BAD9CAD0E9480519B01C9
:108D6000AC01C701B6010E94B3532DA13EA14FA192
:108D700058A50E94E5506B017C01C501B4010E9419
:108D80007E519B01AC01C701B6010E94E152181649
:108D90002CF4F80180829182A282B38280905A0BD7
:108DA00090905B0BA0905C0BB0905D0BD8016D9127
:108DB0007D918D919C910E947E516B017C01EBA174
:108DC000FCA164817581868197810E9480519B01FD
:108DD000AC01C701B6010E94B3532DA13EA14FA122
:108DE00058A50E94E5506B017C01C501B4010E94A9
:108DF0007E519B01AC01C701B6010E94E1521816D9
:108E000034F4D8018D929D92AD92BC9213978090CC
:108E1000620B9090630BA090640BB090650B0BA15C
:108E20001CA10C5B1F4FF8016081718182819381CD
:108E30000E947E516B017C0169966CAD7DAD8EAD5B
:108E40009FAD69970E9480519B01AC01C701B6019B
:108E50000E94B3532DA13EA14FA158A50E94E550F9
:108E60006B017C01C501B4010E947E519B01AC01E4
:108E7000C701B6010E94E152181634F4D8018D9250
:108E80009D92AD92BC92139780905E0B90905F0B79
:108E9000A090600BB090610BF801608171818281BC
:108EA00093810E947E516B017C01ABA1BCA11896FD
:108EB0006D917D918D919C911B970E9480519B019A
:108EC000AC01C701B6010E94B3532DA13EA14FA131
:108ED00058A50E94E5506B017C01C501B4010E94B8
:108EE0007E519B01AC01C701B6010E94E1521816E8
:108EF0002CF4F80180829182A282B382EBA1FCA1C2
:108F0000EC5BFF4F60817181828193810E947E5171
:108F10006B017C01F301A2010F2F162D252F342D9B
:108F2000A90198010E94E550462F572F682F792FED
:108F30006D964CAF5DAF6EAF7FAF6D97ABA1BCA12F
:108F4000D2964D935D936D937C93D597C701B601EF
:108F50002DEB37E346E051E40E94B3530E944D519C
:108F6000DC01CB01EBA1FCA1848F958FA68FB78F7D
:108F70002091720B3091730B4091740B5091750BD3
:108F800069962CAF3DAF4EAF5FAF699749855A8563
:108F90006B857C8549AF5AAF6BAF7CAFCB01BA0113
:108FA00020E030E040E050E00E94E152C9ACDAAC91
:108FB000EBACFCAC181624F0F7FAF094F7F8F09448
:108FC00060916E0B70916F0B8091700B9091710B93
:108FD00025966CAF7DAF8EAF9FAF259720E030E038
:108FE00040E05FE30E94B353162F072FB82EA92E3F
:108FF000C701B601A8019501C52ED42EE32EF22E8D
:10900000A70196010E94E152181684F069966CAD92
:109010007DAD8EAD9FAD699720E030E040E05FE32D
:109020000E94B353162F072FB82EA92EABA1BCA1B7
:1090300092962C90929793963C9093979496BC918D
:10904000BDA3EBA1FCA1F5A1F9A7A8019501852F6E
:10905000902FA32FBA2DBC01CD013DA1C22CD32C42
:10906000E32EFF2EA70196010E94DE5087FD04C06B
:10907000122D032DBE2CAF2C2D853E854F85588992
:1090800029AB3AAB4BAB5CABCA01B90120E030E095
:1090900040E050E00E94E152C9A8DAA8EBA8FCA881
:1090A000181624F0F7FAF094F7F8F09440916A0B50
:1090B00050916B0B60916C0B70916D0B29964CAFBE
:1090C0005DAF6EAF7FAF2997CB01BA0120E030E0F2
:1090D00040E05FE30E94B353962E872E782E692ED0
:1090E000C701B6019401472D562DC32ED22E7A0109
:1090F000A70196010E94E152181684F4A801950177
:10910000852F902FA32FBA2DBC01CD01A701960169
:109110000E94DE5087FD02C0840153016DA97EA923
:10912000623071050CF449C16091C60B7091C70B98
:109130008091C80B9091C90B20E030E040E050E0F6
:109140000E94E15218160CF038C18091B60B909134
:10915000B70BA091B80BB091B90B8DAB9EABAFAB79
:10916000B8AF69817A818B819C812DA93EA94FA9D5
:1091700058AD0E9404509B01AC010E94B353C62E0F
:10918000972E882EF92E4090BA0B5090BB0B609012
:10919000BC0B7090BD0B6D817E818F819885A30182
:1091A00092010E9404509B01AC010E94B353B62F60
:1091B000A72FF82FE92F4C2D592D682D7F2DCB018E
:1091C000BA01AD019F01C52ED42EE32EF22EA701C8
:1091D00096010E9405500E9420546B017C016DA9EC
:1091E0007EA98FA998AD20E030E040E050E00E94D9
:1091F000DE50882351F4C301B20120E030E040E0AA
:1092000050E00E94DE50882321F0122D032DBDA0D6
:10921000A9A4C701B60169962CAD3DAD4EAD5FADB9
:1092200069970E94E1521816D4F469966CAD7DAD31
:109230008EAD9FAD6997A70196010E94E5509B01F5
:10924000AC01F801B5018F2F902FA72FBA2DBC01CB
:10925000CD010E94B353162F072FB82EA92E69AD4A
:109260007AAD8BAD9CAD2091BE0B3091BF0B409180
:10927000C00B5091C10B0E9404504B01782E692EF7
:109280006B01E82EF92E44244394CB01A72DB62D73
:10929000BC01CD0120E030E040E050E00E94E1520E
:1092A00018162CF04424D701C601B05803C0C401DD
:1092B000A72DB62DBC01CD0125962CAD3DAD4EADF3
:1092C0005FAD25970E94E152181604F5442021F461
:1092D000F7FAF094F7F8F09425966CAD7DAD8EAD6D
:1092E0009FAD2597A70196010E94E5509B01AC0117
:1092F000F801B5018F2F902FA72FBA2DBC01CD01FA
:109300000E94B353162F072FB82EA92E69A97AA948
:109310008BA99CA92091C20B3091C30B4091C40B27
:109320005091C50B0E9404504B01782E692E6B01A1
:10933000E82EF92E44244394CB01A72DB62DBC0171
:10934000CD0120E030E040E050E00E94E1521816EC
:109350002CF04424D701C601B05803C0C401A72D86
:10936000B62DBC01CD0129962CAD3DAD4EAD5FAD06
:1093700029970E94E152181604F5442021F4F7FAC7
:10938000F094F7F8F09429966CAD7DAD8EAD9FAD5D
:109390002997A70196010E94E5509B01AC01F801B5
:1093A000B5018F2F902FA72FBA2DBC01CD010E94A0
:1093B000B353162F072FB82EA92EA8019501852F7C
:1093C000902FA32FBA2DEBA1FCA182A793A7A4A74E
:1093D000B5A76D962CAD3DAD4EAD5FAD6D975058B8
:1093E000CA01B9010E94055021962CAD3DAD4EAD8C
:1093F0005FAD21970E94B3539B01AC0160E070E028
:1094000080E890E40E9404500E9420544B01782E82
:10941000692EA8019501852F902FA32FBA2DBC018D
:10942000CD019301C82CD92CE32EF22EA701960171
:109430000E94DE5087FD03C0182D092D5301A8019D
:109440009501852F902FA32FBA2DEBA1FCA186A308
:1094500097A3A0A7B1A73DA129A5822D932DA32F46
:10946000B22FBC01CD019301C82CD92CE32EF62CD0
:10947000A70196010E94DE5018163CF081E0ABA1D6
:10948000BCA1D7968C93D79703C0EBA1FCA117AAD8
:1094900081E0ABA1BCA1D6968C93A6EBBBE0FE010C
:1094A000319680E101900D928150E1F73DA129A50F
:1094B000822D932DA32FB22F8093C60B9093C70BB1
:1094C000A093C80BB093C90BA8019501852F902FCD
:1094D000A32FBA2DBC01CD015DA149A5022D132DED
:1094E000252F342FA90198010E94E5506B017C01C2
:1094F00060E070E080E090E45DA149A5252F342F65
:10950000A90198010E94E5508B019C018BA19CA1AF
:10951000B701A6010E94F33A6E96BFAD6E97B09365
:1095200075062D962CAD3DAD4EAD5FAD2D972093BC
:10953000460B3093470B4093480B5093490B619671
:109540004CAD5DAD6EAD7FAD619740934A0B5093CE
:109550004B0B60934C0B70934D0B65966CAD7DADD2
:109560008EAD9FAD659760934E0B70934F0B8093BC
:10957000500B9093510B8DA59EA5AFA5B8A98093D4
:10958000520B9093530BA093540BB093550B0E9426
:10959000233F0E942809CF59DF4F0FB6F894DEBF52
:1095A0000FBECDBFDF91CF911F910F91FF90EF9034
:1095B000DF90CF90BF90AF909F908F907F906F90F3
:1095C0005F904F903F902F900895AF92BF92CF92AF
:1095D000DF92EF92FF920F931F93CF93DF93EB01F4
:1095E0006A015901FC01608171818281938120911E
:1095F000920B3091930B4091940B5091950B0E94DC
:10960000B3530E948353A6E4EA2EABE0FA2E609394
:10961000460B7093470B8093480B9093490B6881DE
:1096200079818A819B812091960B3091970B409193
:10963000980B5091990B0E94B3530E94835387015A
:109640000C5F1F4F60934A0BF801718382839383F1
:10965000F601608171818281938120919A0B309112
:109660009B0B40919C0B50919D0B0E94B3530E9409
:109670008353E701289660934E0B79838A839B83FB
:10968000F501608171818281938120919E0B3091DF
:109690009F0B4091A00B5091A10B0E94B3530E94CD
:1096A0008353F7013C966093520B718382839383BB
:1096B000C701B801AE019F010E946B1080E090E0ED
:1096C000A0E0B0E08093C60B9093C70BA093C80BAB
:1096D000B093C90B8093B60B9093B70BA093B80BC4
:1096E000B093B90B8093BA0B9093BB0BA093BC0BB8
:1096F000B093BD0B8093BE0B9093BF0BA093C00B98
:10970000B093C10B8093C20B9093C30BA093C40B77
:10971000B093C50BDF91CF911F910F91FF90EF9008
:10972000DF90CF90BF90AF900895FC016081718170
:109730008281938120919E0B30919F0B4091A00BD1
:109740005091A10B0E94B3530E9483536093520B1C
:109750007093530B8093540B9093550B82E59BE0D1
:109760000E94A71008958093730608951F920F9288
:109770000FB60F920BB60F9211242F933F934F9376
:109780005F936F937F938F939F93AF93BF93EF9369
:10979000FF938091CE0B9091CF0B009729F0E09131
:1097A000CE0BF091CF0B1995FF91EF91BF91AF9137
:1097B0009F918F917F916F915F914F913F912F91E9
:1097C0000F900BBE0F900FBE0F901F9018951F9219
:1097D0000F920FB60F920BB60F9211242F933F9357
:1097E0004F935F936F937F938F939F93AF93BF93A9
:1097F000EF93FF938091D00B9091D10B009729F0BC
:10980000E091D00BF091D10B1995FF91EF91BF91A1
:10981000AF919F918F917F916F915F914F913F9108
:109820002F910F900BBE0F900FBE0F901F901895A9
:109830001F920F920FB60F920BB60F9211242F9317
:109840003F934F935F936F937F938F939F93AF93C8
:10985000BF93EF93FF938091D20B9091D30B00971E
:1098600029F0E091D20BF091D30B1995FF91EF9174
:10987000BF91AF919F918F917F916F915F914F9128
:109880003F912F910F900BBE0F900FBE0F901F9026
:1098900018951F920F920FB60F920BB60F921124CC
:1098A0002F933F934F935F936F937F938F939F93E8
:1098B000AF93BF93EF93FF938091D40B9091D50B0F
:1098C000009729F0E091D40BF091D50B1995FF91F9
:1098D000EF91BF91AF919F918F917F916F915F9128
:1098E0004F913F912F910F900BBE0F900FBE0F9095
:1098F0001F9018951F920F920FB60F920BB60F92F2
:1099000011242F933F934F935F936F937F938F9384
:109910009F93AF93BF93EF93FF938091CA0B909166
:10992000CB0B009729F0E091CA0BF091CB0B199566
:10993000FF91EF91BF91AF919F918F917F916F9127
:109940005F914F913F912F910F900BBE0F900FBEE3
:109950000F901F9018951F920F920FB60F920BB693
:109960000F9211242F933F934F935F936F937F93A5
:109970008F939F93AF93BF93EF93FF938091CC0B03
:109980009091CD0B009729F0E091CC0BF091CD0B8D
:109990001995FF91EF91BF91AF919F918F917F9119
:1099A0006F915F914F913F912F910F900BBE0F9050
:1099B0000FBE0F901F9018951F920F920FB60F9227
:1099C0000BB60F9211242F933F934F935F936F9396
:1099D0007F938F939F93AF93BF93EF93FF93809168
:1099E000D60B9091D70B009729F0E091D60BF09110
:1099F000D70B1995FF91EF91BF91AF919F918F91E7
:109A00007F916F915F914F913F912F910F900BBE7E
:109A10000F900FBE0F901F9018951F920F920FB6C8
:109A20000F920BB60F9211242F933F934F935F9396
:109A30006F937F938F939F93AF93BF93EF93FF9316
:109A40008091D80B9091D90B009729F0E091D80B19
:109A5000F091D90B1995FF91EF91BF91AF919F9123
:109A60008F917F916F915F914F913F912F910F90C7
:109A70000BBE0F900FBE0F901F9018951F93CF93A2
:109A8000DF93182FEB0161E00E948E4E209711F4B6
:109A9000812FC7C0CF3FD10511F4812FC4C0E12F62
:109AA000F0E0ED5DF04FE491E93009F466C0EA3092
:109AB000B0F4E430F1F1E53040F4E23059F1E33054
:109AC00070F5E13009F0A9C020C0E73009F443C0C7
:109AD000E83008F048C0E63009F09FC034C0ED30EF
:109AE00009F473C0EE3038F4EB3009F45AC0EC30AE
:109AF00008F061C04CC0E03109F47BC0E13109F4E9
:109B000082C0EF3009F089C06AC084B5806884BD26
:109B1000C7BD8CC084B5806284BDC8BD87C080913C
:109B20008000806880938000D0938900C093880073
:109B30007DC080918000806280938000D0938B00F4
:109B4000C0938A0073C08091B00080688093B00099
:109B5000C093B3006BC08091B00080628093B0006E
:109B6000C093B40063C0809190008068809390009F
:109B7000D0939900C093980059C080919000806262
:109B800080939000D0939B00C0939A004FC0809127
:109B90009000886080939000D0939D00C0939C00BB
:109BA00045C08091A00080688093A000D093A90058
:109BB000C093A8003BC08091A00080628093A00069
:109BC000D093AB00C093AA0031C08091A000886000
:109BD0008093A000D093AD00C093AC0027C08091CB
:109BE0002001806880932001D0932901C09328012F
:109BF0001DC080912001806280932001D0932B01B1
:109C0000C0932A0113C080912001886080932001B5
:109C1000D0932D01C0932C0109C0812FC038D105EC
:109C200014F460E001C061E00E94AF4EDF91CF917B
:109C30001F910895893009F449C08A30A0F4843016
:109C400051F1853040F4823079F1833000F5813074
:109C500009F063C026C0873079F1883098F58630E6
:109C600009F05BC025C08D3009F442C08E3028F465
:109C70008B30B1F18C30C0F52DC0803109F442C079
:109C8000813109F445C08F3009F047C037C0809159
:109C900080008F7703C0809180008F7D809380004B
:109CA000089584B58F7702C084B58F7D84BD0895F3
:109CB0008091B0008F7703C08091B0008F7D80933A
:109CC000B0000895809190008F7707C08091900038
:109CD0008F7D03C080919000877F809390000895CE
:109CE0008091A0008F7707C08091A0008F7D03C076
:109CF0008091A000877F8093A0000895809120012B
:109D00008F7703C0809120018F7D8093200108957B
:109D100080912001877F80932001089590E0FC01CD
:109D2000E759F04F2491FC01E155F04FE491EE2307
:109D3000A9F0F0E0EE0FFF1FE75DFF4E85919491D3
:109D4000DC019FB7F8948C91662329F42095822337
:109D50008C939FBF0895822B8C939FBF08950F9380
:109D60001F93CF93DF930F92CDB7DEB7282F30E04C
:109D7000F901ED5DF04F8491F901E759F04F14912D
:109D8000F901E155F04F04910023D1F0882321F02F
:109D900069830E941A4E6981E02FF0E0EE0FFF1FE9
:109DA000E15FFF4E85919491DC019FB7F8948C910F
:109DB000662319F41095812301C0812B8C939FBFDA
:109DC0000F90DF91CF911F910F9108951F920F92E5
:109DD0000FB60F9211242F933F938F939F93AF93BE
:109DE000BF938091DA0B9091DB0BA091DC0BB091CB
:109DF000DD0B3091E20B232F2D5F2D3720F40196E0
:109E0000A11DB11D05C0232F2A570296A11DB11D0A
:109E10002093E20B8093DA0B9093DB0BA093DC0B87
:109E2000B093DD0B8091DE0B9091DF0BA091E00BE6
:109E3000B091E10B0196A11DB11D8093DE0B9093B3
:109E4000DF0BA093E00BB093E10BBF91AF919F911B
:109E50008F913F912F910F900FBE0F901F901895EB
:109E60000F931F938FB7F8940091DA0B1091DB0BCF
:109E70002091DC0B3091DD0B8FBFB801C9011F9120
:109E80000F9108950F931F939FB7F8940091DE0BE5
:109E90001091DF0B2091E00B3091E10B86B5A89B70
:109EA00006C08F3F21F00F5F1F4F2F4F3F4F9FBFC7
:109EB000322F212F102F0027080F111D211D311DBA
:109EC00042E0000F111F221F331F4A95D1F7B8013E
:109ED000C9011F910F910895CF92DF92EF92FF92E7
:109EE000CF93DF936B017C010E94424FDC01CB01D9
:109EF000EC010FC00E94424F6C1B7D0B83E0683E5B
:109F0000780738F00894C108D108E108F108C85171
:109F1000DC4FC114D104E104F10461F7DF91CF916A
:109F2000FF90EF90DF90CF900895789484B5826091
:109F300084BD84B5816084BD85B5826085BD85B5ED
:109F4000816085BDEEE6F0E0808181608083E1E89C
:109F5000F0E01082808182608083808181608083D4
:109F6000E0E8F0E0808181608083E1EBF0E08081D7
:109F700084608083E0EBF0E0808181608083E1E9B0
:109F8000F0E0808182608083808181608083E0E96D
:109F9000F0E0808181608083E1EAF0E0808182608E
:109FA0008083808181608083E0EAF0E0808181604D
:109FB0008083E1E2F1E08081826080838081816042
:109FC0008083E0E2F1E0808181608083EAE7F0E075
:109FD00080818460808380818260808380818160D1
:109FE00080838081806880831092C10008950E94E0
:109FF000954F0E94BC2DC0E0D0E00E948D2D20978F
:10A00000E1F30E940000F9CF5058BB27AA270ED0D9
:10A0100076C23FD230F044D220F031F49F3F11F4A9
:10A020001EF40FC20EF4E095E7FBDCC1E92F89D2E4
:10A0300080F3BA17620773078407950718F071F465
:10A040009EF5B8C20EF4E0950B2EBA2FA02D0B0191
:10A05000B90190010C01CA01A0011124FF27591B6D
:10A0600099F0593F50F4503E68F11A16F040A22F73
:10A07000232F342F4427585FF3CF469537952795E4
:10A08000A795F0405395C9F77EF41F16BA0B620BE3
:10A09000730B840BBAF09150A1F0FF0FBB1F661F2A
:10A0A000771F881FC2F70EC0BA0F621F731F841F6D
:10A0B00048F4879577956795B795F7959E3F08F093
:10A0C000B3CF9395880F08F09927EE0F9795879552
:10A0D0000895DFD158F080E891E009F49EEFE0D1D7
:10A0E00028F040E851E059F45EEF09C0AAC162C20D
:10A0F000E92FE07826D268F3092E052AC1F3261746
:10A1000037074807590738F00E2E07F8E02569F0A1
:10A11000E025E0640AC0EF6307F8009407FADB016A
:10A12000B9019D01DC01CA01AD01EF935DD0E7D11A
:10A130000AD05F91552331F02BED3FE049E450FD0B
:10A1400049EC63CF0895DF93DD27B92FBF7740E84F
:10A150005FE31616170648075B0710F4D92F96D24F
:10A160009F938F937F936F93A9D3E4EEF0E06CD12C
:10A17000C6D12F913F914F915F9101D3DD2349F0DB
:10A180009058A2EA2AED3FE049EC5FE3D0785D27E2
:10A190004DDFDF91B4C1F7D180F09F3740F49111CA
:10A1A0000EF409C260E070E080E89FE3089526F0B5
:10A1B0001B16611D711D811D1BC135C1EFD008F437
:10A1C00081E0089575D1E395ABC10CD098C168D1F9
:10A1D00040F05FD130F021F45F3F19F003C151111D
:10A1E000EAC12FC1AED198F39923C9F35523B1F336
:10A1F000951B550BBB27AA2762177307840738F0F6
:10A200009F5F5F4F220F331F441FAA1FA9F333D054
:10A210000E2E3AF0E0E830D091505040E695001C08
:10A22000CAF729D0FE2F27D0660F771F881FBB1FC4
:10A23000261737074807AB07B0E809F0BB0B802D9E
:10A24000BF01FF2793585F4F2AF09E3F510568F0EA
:10A25000C9C0B1C15F3FECF3983EDCF386957795BA
:10A260006795B795F7959F5FC9F7880F911D9695EC
:10A27000879597F90895E1E0660F771F881FBB1F48
:10A28000621773078407BA0720F0621B730B840BF5
:10A29000BA0BEE1F88F7E095089504D06894B111C9
:10A2A0008AC1089556D188F09F5790F0B92F992709
:10A2B000B751A0F0D1F0660F771F881F991F1AF0D1
:10A2C000BA95C9F712C0B13081F074D1B1E00895E8
:10A2D00071C1672F782F8827B85F39F0B93FCCF369
:10A2E000869577956795B395D9F73EF490958095C7
:10A2F000709561957F4F8F4F9F4F0895E89409C0E7
:10A3000097FB3EF490958095709561957F4F8F4FA8
:10A310009F4F9923A9F0F92F96E9BB279395F695BE
:10A32000879577956795B795F111F8CFFAF4BB0F3C
:10A3300011F460FF1BC06F5F7F4F8F4F9F4F16C0A0
:10A34000882311F096E911C0772321F09EE8872F2A
:10A35000762F05C0662371F096E8862F70E060E0E6
:10A360002AF09A95660F771F881FDAF7880F96955F
:10A37000879597F9089507D180F09F3740F49111A0
:10A380000EF019C160E070E080E89FEB089526F4BC
:10A390001B16611D711D811D2BC045C0990F000842
:10A3A000550FAA0BE0E8FEEF16161706E807F907A7
:10A3B000C0F012161306E407F50798F0621B730B42
:10A3C000840B950B39F40A2661F0232B242B252BC3
:10A3D00021F408950A2609F4A140A6958FEF811D66
:10A3E000811D089597F99F6780E870E060E0089507
:10A3F000882371F4772321F09850872B762F07C09C
:10A40000662311F499270DC09051862B70E060E00F
:10A410002AF09A95660F771F881FDAF7880F9695AE
:10A42000879597F908959F3F31F0915020F48795D3
:10A4300077956795B795880F911D9695879597F9AC
:10A4400008959FEF80EC0895DF93CF931F930F93B0
:10A45000FF92EF92DF927B018C01689405C0DA2EA7
:10A46000EF018DD1FE01E894A5912591359145919B
:10A470005591AEF3EF01DADDFE019701A801DA9400
:10A4800079F7DF90EF90FF900F911F91CF91DF91BF
:10A49000089500240A94161617061806090608954A
:10A4A00000240A9412161306140605060895C9CF4F
:10A4B00050D0E8F3E894E0E0BB279F57F0F02AED96
:10A4C0003FE049EC06C0EE0FBB0F661F771F881FE9
:10A4D00028F0B23A62077307840728F0B25A620B79
:10A4E000730B840BE3959A9572F7803830F49A9544
:10A4F000BB0F661F771F881FD2F7904896CF092E93
:10A500000394000C11F4882352F0BB0F40F4BF2BCE
:10A5100011F460FF04C06F5F7F4F8F4F9F4F08950E
:10A52000EF93E0FF06C0A2EA2AED3FE049EC5FEBC3
:10A530007DDDE5DF0F90039401FC9058E1E1F1E04F
:10A54000C7C157FD9058440F551F59F05F3F71F038
:10A550004795880F97FB991F61F09F3F79F087958A
:10A560000895121613061406551FF2CF4695F1DF13
:10A5700008C0161617061806991FF1CF86957105A3
:10A58000610508940895E5DFA0F0BEE7B91788F4E7
:10A59000BB279F3860F41616B11D672F782F8827C8
:10A5A000985FF7CF869577956795B11D9395963906
:10A5B000C8F30895E894BB2766277727CB0197F95E
:10A5C0000895ECDE08F48FEF089563DF19F068DF7B
:10A5D00009F037CF07CFB901CA0125CF9F775F7741
:10A5E000B0DF98F39923B9F35523B9F3FF279517F3
:10A5F00058F4E52FE91BED3070F75E3B10F0F1E405
:10A600001CC09034E0F40AC0E92FE51BED3028F7B8
:10A610009E3B10F0F1E411C0503488F4F9EA88232D
:10A620002AF09A95660F771F881FDAF744232AF0DD
:10A630005A95220F331F441FDAF79F1B5F1BFF93AE
:10A640001F930F93FF92EF9279018A01BB27AB2FE3
:10A650009B01AC0196D09701A801BF937B018C01AF
:10A66000AA27BA2FB901CA018CD0AF919701A801CE
:10A67000EF90FF900F911F91D9DC41DFE1D04F9116
:10A6800040FF0895552747FD509509C09B01AC0137
:10A6900060E070E080E89FE398CDA4CEC4CE59DF9F
:10A6A000E8F39923D9F3940F511DBBF39150504017
:10A6B00094F059F0882332F0660F771F881F91506D
:10A6C0005040C1F79E3F510544F7880F911D969564
:10A6D000879597F908955F3FACF0983E9CF0BB27B3
:10A6E000869577956795B79508F4B1609395C1F70E
:10A6F000BB0F58F711F460FFE8CF6F5F7F4F8F4FAC
:10A700009F4FE3CF58CF25DF58F19E5758F198510E
:10A71000A0F0E9F0983020F5092E9927660F771FF1
:10A72000881F991F0A94D1F712C0062E672F782F21
:10A730008827985F11F4000C07C0993FB4F3869501
:10A74000779567959395D9F7611D711D811D3EF42D
:10A7500090958095709561957F4F8F4F9F4F08958D
:10A76000689429CF27CF0BD0CACE93DE28F098DE8D
:10A7700018F0952309F036CE64CE11241CCFE1DE0B
:10A78000A0F3959FD1F3950F50E0551F629FF00104
:10A79000729FBB27F00DB11D639FAA27F00DB11D5D
:10A7A000AA1F649F6627B00DA11D661F829F2227E6
:10A7B000B00DA11D621F739FB00DA11D621F839F6D
:10A7C000A00D611D221F749F3327A00D611D231F43
:10A7D000849F600D211D822F762F6A2F11249F5791
:10A7E00050408AF0E1F088234AF0EE0FFF1FBB1FB4
:10A7F000661F771F881F91505040A9F79E3F510553
:10A8000070F0F0CDD8CE5F3FECF3983EDCF3869548
:10A8100077956795B795F795E7959F5FC1F7FE2BFD
:10A82000880F911D9695879597F908959F9340DE1F
:10A830000F9007FCEE5F74CE11F40EF402CEF3CD50
:10A8400088DED0F39923D9F3CEF39F57550B87FFBA
:10A8500038D00024A0E640EA90018058569597959C
:10A8600028F4805C660F771F881F20F026173707B3
:10A87000480730F4621B730B840B202931294A2BC3
:10A88000A69517940794202531254A2758F7660F77
:10A89000771F881F20F026173707480730F4620B10
:10A8A000730B840B200D311D411DA09581F7B9015B
:10A8B000842F9158880F9695879508959B01AC0138
:10A8C00052CF91505040660F771F881FD2F70895DE
:10A8D0009F938F937F936F93FF93EF939B01AC01B3
:10A8E00042DFEF91FF91B0DD2F913F914F915F914A
:10A8F0003ACF629FD001739FF001829FE00DF11D5E
:10A90000649FE00DF11D929FF00D839FF00D749FE9
:10A91000F00D659FF00D9927729FB00DE11DF91F95
:10A92000639FB00DE11DF91FBD01CF0111240895F2
:10A9300097FB092E07260AD077FD04D049D006D010
:10A9400000201AF4709561957F4F0895F6F7909561
:10A9500081959F4F0895A1E21A2EAA1BBB1BFD01F2
:10A960000DC0AA1FBB1FEE1FFF1FA217B307E407EE
:10A97000F50720F0A21BB30BE40BF50B661F771F46
:10A98000881F991F1A9469F7609570958095909526
:10A990009B01AC01BD01CF01089597FB092E05264F
:10A9A0000ED057FD04D0D7DF0AD0001C38F45095E4
:10A9B0004095309521953F4F4F4F5F4F0895F6F7E3
:10A9C00090958095709561957F4F8F4F9F4F08951B
:10A9D000AA1BBB1B51E107C0AA1FBB1FA617B707C5
:10A9E00010F0A61BB70B881F991F5A95A9F78095E1
:10A9F0009095BC01CD0108956F927F928F929F92A6
:10AA0000AF92BF92CF92DF92EF92FF920F931F937C
:10AA1000CF93DF935B016115710521F0DB018C930E
:10AA200011969C937C01E7010894E11CF11C0881BC
:10AA30006701802F90E00E94BA570097A1F70D326E
:10AA400041F4098142E0C42ED12CCC0EDD1E11E070
:10AA500009C00B3231F4098132E0C32ED12CCC0E67
:10AA6000DD1E10E0E6012197CE0163E470E143E0D2
:10AA700050E00E94C2570097D1F4E6012296CE0121
:10AA800066E470E145E050E00E94C257009711F47F
:10AA9000E6012796A114B10419F0F501D183C08312
:10AAA00030E020E090E8112309F40DC107C1CE0188
:10AAB0006BE470E143E050E00E94C257009759F404
:10AAC000A114B10409F4FCC0C6010296D501119687
:10AAD0009C938E93F5C040E050E060E070E08824E5
:10AAE000992400530A3090F51260212F30E0C901FB
:10AAF0008870907012FF06C0009769F50894811C59
:10AB0000911C29C0009719F0089481089108DB0175
:10AB1000CA01D2E0880F991FAA1FBB1FDA95D1F78F
:10AB2000480F591F6A1F7B1F440F551F661F771F51
:10AB3000400F511D611D711D4839B9E95B07B9E925
:10AB40006B07B9E17B0738F0146005C00E3F39F49C
:10AB500013FD43C01860F60101916F01C2CF0533A8
:10AB600011F00531D1F5D601EC91ED3211F41061FF
:10AB700008C0EB3229F0C601019621E030E008C0A0
:10AB8000D6011196EC911197C601029622E030E0B1
:10AB9000E053EA3020F06C01C21AD30A1EC0DC0177
:10ABA00020E030E0FCE020383F075CF4C901880F6A
:10ABB000991F880F991F280F391F220F331F2E0F3F
:10ABC000311DED91E0536D01EA3060F314FF03C0D5
:10ABD000309521953F4F820E931EC12FD0E011FF7B
:10ABE00008C0A114B10429F0C6010197D5018D93C5
:10ABF0009C93CB01BA010E947E516B017C01CE0176
:10AC0000837090708330910521F4F7FAF094F7F88F
:10AC1000F094C701B60120E030E040E050E00E942F
:10AC2000DE50882309F445C097FE07C090948194B4
:10AC300091089394CAE7D0E102C0C2E6D0E198EE51
:10AC4000692E9FEF792E6C0E7D1E20E2A22EB12C74
:10AC50000FC0FE010591159125913491C701B601F0
:10AC6000A90198010E94B3536B017C018A189B08CB
:10AC70008A149B0474F72497B594A794C615D70536
:10AC8000B9F7C601D7012A2F220F2B2F221F2F3FE2
:10AC900051F0BC01CD0120E030E040E050E00E94E6
:10ACA000DE50882331F482E290E09093E80B8093A9
:10ACB000E70B3C2D2D2D9E2D8F2D06C08FEF04C050
:10ACC00030E020E090EC8FE7B901AC01872F922FA4
:10ACD000A52FB42FBC01CD01DF91CF911F910F9112
:10ACE000FF90EF90DF90CF90BF90AF909F908F90AC
:10ACF0007F906F9008952F923F924F925F926F9244
:10AD00007F928F929F92BF92CF92DF92EF92FF92AB
:10AD10000F931F93CF93DF933B018A016115710558
:10AD200019F0FB01808391830115110539F0980119
:10AD3000225030402332310508F004C16C01760105
:10AD40000894C11CD11CF701C08146018C2F90E0F2
:10AD50000E94BA57009799F7CD3249F4F701C181A3
:10AD6000B2E08B2E912C8E0C9F1CD1E00AC0CB320E
:10AD700039F4F701C181A2E08A2E912C8E0C9F1C20
:10AD8000D0E00115110519F000311105C1F4C033EF
:10AD900081F4F4018081883711F0883551F4F40191
:10ADA000C18182E090E0880E991ED26000E110E03F
:10ADB00006C00115110519F4C033C1F422C00830D2
:10ADC0001105F9F00930110524F40230110509F5D7
:10ADD00007C00A30110551F000311105D1F427C028
:10ADE000C12CD12CE12C70E4F72E26C00AE010E033
:10ADF0006CECC62E6CECD62E6CECE62E6CE0F62ECF
:10AE00001BC008E010E0C12CD12CE12C50E1F52E44
:10AE100013C09801442737FD4095542F60E070E03F
:10AE200080E090E80E94AB5469017A0105C0C12C12
:10AE3000D12CE12C48E0F42E20E040E050E060E02E
:10AE400070E01801442437FC4094542C30EDB32EAC
:10AE5000BC0E99E09B1570F48C2F81548A3118F444
:10AE600099ECB92E06C08C2F81568A3150F589EAAB
:10AE7000B82EBC0E8B2D90E08017910714F527FD9E
:10AE80001CC0C416D506E606F706A0F0CB01BA0131
:10AE9000A20191010E947954AB01BC014B0D511DDF
:10AEA000611D711D4130E0E05E07E0E06E07E0E803
:10AEB0007E0710F02FEF01C021E0F401C1914F0196
:10AEC000C5CF6114710489F0222339F008948108F8
:10AED0009108F3019182808208C0D1FF1AC0C40199
:10AEE0000297F3019183808314C027FF12C0D0FF23
:10AEF00005C040E050E060E070E804C04FEF5FEF55
:10AF00006FEF7FE782E290E09093E80B8093E70B8E
:10AF100016C0D0FF08C070956095509541955F4F61
:10AF20006F4F7F4F0CC077FF0AC082E290E0909392
:10AF3000E80B8093E70B4FEF5FEF6FEF7FE78A013E
:10AF40009B0104C000E010E020E030E0B801C9013E
:10AF5000DF91CF911F910F91FF90EF90DF90CF90F5
:10AF6000BF909F908F907F906F905F904F903F9099
:10AF70002F90089591119EC2803219F0895085500A
:10AF8000D0F70895FB01DC014150504088F08D91CD
:10AF900081341CF08B350CF4805E659161341CF0BB
:10AFA0006B350CF4605E861B611171F3990B08958B
:10AFB000881BFCCFFC018191861721F08823D9F7EB
:10AFC000992708953197CF010895FB01DC01415085
:10AFD000504030F08D910190801919F40020B9F79C
:10AFE000881B990B0895FB0151915523A9F0BF01CE
:10AFF000DC014D9145174111E1F759F4CD01019064
:10B00000002049F04D9140154111C9F3FB01411158
:10B01000EFCF81E090E0019708950F931F93CF93B6
:10B02000DF93CDB7DEB72E970FB6F894DEBF0FBE15
:10B03000CDBF0E891F8986E08C831A8309838FEF29
:10B040009FE79E838D83AE01465E5F4FCE010196E2
:10B05000688D798D0E943C58EF81F885E00FF11FD3
:10B0600010822E960FB6F894DEBF0FBECDBFDF91D3
:10B07000CF911F910F9108952F923F924F925F921F
:10B080006F927F928F929F92AF92BF92CF92DF92F8
:10B09000EF92FF920F931F93CF93DF93CDB7DEB75D
:10B0A0002D970FB6F894DEBF0FBECDBF3C017D8754
:10B0B0006C875A01FC0117821682838181FFC9C106
:10B0C0003FE3C32E2E010894411C511CF3019381D0
:10B0D000EC85FD8593FD859193FF8191FD87EC873C
:10B0E000882309F4B2C1853241F493FD859193FF21
:10B0F0008191FD87EC87853229F490E0B3010E94AD
:10B10000735AE4CFEE24DD2410E01032B0F48B3219
:10B1100069F08C3228F4803251F0833271F40BC024
:10B120008D3239F0803349F411602CC01260146004
:10B1300029C0186027C0106125C017FD2EC0282F18
:10B1400020532A3098F416FF08C08E2D880FE82E61
:10B15000EE0CEE0CE80EE20E15C08D2D880FD82EE9
:10B16000DD0CDD0CD80ED20E10620CC08E3221F434
:10B1700016FD6BC1106406C08C3611F4106802C055
:10B18000883659F4EC85FD8593FD859193FF819177
:10B19000FD87EC87882309F0B8CF982F955493301A
:10B1A00018F09052933030F424E030E0A20EB31E39
:10B1B000C9820FC0833631F0833781F0833509F0BF
:10B1C0005AC022C0F5018081898322E030E0A20EBE
:10B1D000B31E21E0E22EF12C420114C092E0292E90
:10B1E000312C2A0C3B1CF5018080918016FF03C096
:10B1F0006E2D70E002C06FEF7FEFC4010E94685AAD
:10B200007C0151011F7715C082E0282E312C2A0CB9
:10B210003B1CF5018080918016FF03C06E2D70E00D
:10B2200002C06FEF7FEFC4010E945D5A7C0110687D
:10B23000510113FD1CC006C080E290E0B3010E94E2
:10B24000735ADA948D2D90E0E816F906A8F30FC032
:10B25000F40117FD859117FF81914F0190E0B30133
:10B260000E94735AD110DA940894E108F108E114AD
:10B27000F10471F7E7C0843611F0893651F5F50114
:10B2800017FF07C080819181A281B38124E030E063
:10B2900008C080819181AA2797FDA095BA2F22E04E
:10B2A00030E0A20EB31E012F0F76B7FF08C0B09595
:10B2B000A095909581959F4FAF4FBF4F0068BC01FF
:10B2C000CD01A2012AE030E00E949F5AF82EF41826
:10B2D0003FC0853721F41F7E2AE030E020C0197F6F
:10B2E0008F36A9F0803720F4883509F0AEC00BC046
:10B2F000803721F0883709F0A8C001C0106114FF21
:10B3000009C0146007C014FF08C0166006C028E01A
:10B3100030E005C020E130E002C020E132E0F5017C
:10B3200017FF07C0608171818281938144E050E002
:10B3300006C06081718180E090E042E050E0A40EA0
:10B34000B51EA2010E949F5AF82EF418012F0F7704
:10B3500006FF09C00E7FFE1430F404FF06C002FD94
:10B3600004C00F7E02C01F2D01C01E2D802F90E053
:10B3700004FF0CC0FE01EF0DF11D2081203311F4FC
:10B38000097E09C002FF06C01E5F05C08678907066
:10B39000009709F01F5F802E992403FD12C000FF63
:10B3A0000DC0EF2C1D1550F4ED0CE11A1D2D06C03B
:10B3B00080E290E0B3010E94735A1F5F1D15C0F335
:10B3C00004C01D1510F4D11A01C0DD2484FE0FC085
:10B3D00080E390E0B3010E94735A82FE1FC081FE99
:10B3E00003C088E590E010C088E790E00DC0C4017C
:10B3F00086789070009791F081FC02C080E201C0D5
:10B400008BE207FD8DE290E0B3010E94735A06C003
:10B4100080E390E0B3010E94735AEA94FE14C0F3F3
:10B42000FA94F201EF0DF11D808190E0B3010E94CA
:10B43000735AFF20A9F706C080E290E0B3010E9492
:10B44000735ADA94DD20C1F741CEF30186819781EA
:10B4500002C08FEF9FEF2D960FB6F894DEBF0FBEA0
:10B46000CDBFDF91CF911F910F91FF90EF90DF90B3
:10B47000CF90BF90AF909F908F907F906F905F9094
:10B480004F903F902F900895F999FECF92BD81BDC6
:10B49000F89A992780B50895262FF999FECF1FBAFB
:10B4A00092BD81BD20BD0FB6F894FA9AF99A0FBEED
:10B4B00001960895992788270895FC010590615009
:10B4C00070400110D8F7809590958E0F9F1F0895BA
:10B4D000FC016150704001900110D8F78095909563
:10B4E0008E0F9F1F08950F931F93CF93DF938C01AF
:10B4F000EB018B8181FF1BC082FF0DC02E813F813C
:10B500008C819D812817390764F4E881F9810193C2
:10B51000F983E88306C0E885F985802F199500979F
:10B5200031F48E819F8101969F838E8302C00FEF3D
:10B530001FEFC801DF91CF911F910F910895FA017C
:10B54000AA27283051F1203181F1E8946F936E7F62
:10B550006E5F7F4F8F4F9F4FAF4FB1E03ED0B4E053
:10B560003CD0670F781F891F9A1FA11D680F791F94
:10B570008A1F911DA11D6A0F711D811D911DA11DA5
:10B5800020D009F468943F912AE0269F11243019B5
:10B59000305D3193DEF6CF010895462F4770405D50
:10B5A0004193B3E00FD0C9F7F6CF462F4F70405DFF
:10B5B0004A3318F0495D31FD4052419302D0A9F75A
:10B5C000EACFB4E0A6959795879577956795BA9554
:10B5D000C9F700976105710508959B01AC010A2E1A
:10B5E00006945795479537952795BA95C9F7620FF1
:0EB5F000731F841F951FA01D0895F894FFCFB0
:10B5FE00537465707261746520746F206869676832
:10B60E00203A20004D313130005573696E67204469
:10B61E00656661756C742073657474696E67733AD0
:10B62E0000FB7A9D42FB7A9D4255550544D57858CC
:10B63E004400007A4300007A430000A0400000342A
:10B64E004228230000282300006400000010270079
:10B65E00004820004C20002569206D696E2C2025A5
:10B66E006920736563004D31303420496E76616C0C
:10B67E00696420657874727564657220004D31308E
:10B68E003520496E76616C696420657874727564D4
:10B69E00657220004D31303920496E76616C6964D7
:10B6AE0020657874727564657220003F006F6B00C0
:10B6BE0020703A0020693A0020643A0020633A0074
:10B6CE005400496E76616C69642065787472756495
:10B6DE00657200416374697665204578747275648D
:10B6EE0065723A20002E0001010101016400640020
:10B6FE0000803B4500803B45000070430000000089
:10B70E000080BB440160EA00000000803FFF5B4107
:10B71E00440BD7233E9A99B141FF3F0158595A45E0
:10B72E0000000100190017001B00160018001F0072
:10B73E0021001D001A001C002500270023001E00FA
:10B74E0020000D000C00040007002B002D00290026
:0AB75E00020008000900FFFF0A00C6
:00000001FF
